ARM GAS  /tmp/ccNMEBpy.s 			page 1


   1              		.cpu cortex-m4
   2              		.eabi_attribute 27, 1
   3              		.eabi_attribute 28, 1
   4              		.eabi_attribute 20, 1
   5              		.eabi_attribute 21, 1
   6              		.eabi_attribute 23, 3
   7              		.eabi_attribute 24, 1
   8              		.eabi_attribute 25, 1
   9              		.eabi_attribute 26, 1
  10              		.eabi_attribute 30, 1
  11              		.eabi_attribute 34, 1
  12              		.eabi_attribute 18, 4
  13              		.file	"timers.c"
  14              		.text
  15              	.Ltext0:
  16              		.cfi_sections	.debug_frame
  17              		.section	.text.MX_TIM17_Init,"ax",%progbits
  18              		.align	1
  19              		.arch armv7e-m
  20              		.syntax unified
  21              		.thumb
  22              		.thumb_func
  23              		.fpu fpv4-sp-d16
  25              	MX_TIM17_Init:
  26              	.LFB341:
  27              		.file 1 "Core/Src/timers.c"
   1:Core/Src/timers.c **** #include "timers.h"
   2:Core/Src/timers.c **** #include "temperature.h"
   3:Core/Src/timers.c **** #define   TIM_GLOBAL_PRESCALER 1 // frequency = 40Mhz
   4:Core/Src/timers.c **** #define   TIM_TRIGGER_PERIOD 299 // 10us
   5:Core/Src/timers.c **** #define   TIM_TRIGGER_COMPARE 39 // 2us
   6:Core/Src/timers.c **** #define   TIM_DISCHARGE_PERIOD 189 // 5us
   7:Core/Src/timers.c **** #define   TIM_DISCHARGE_PULSE 139 // 4us
   8:Core/Src/timers.c **** 
   9:Core/Src/timers.c **** #define TIM_TEMP_PRESCALER 39999 // 2kHz
  10:Core/Src/timers.c **** #define TIM_TEMP_PERIOD 20000 // 10s
  11:Core/Src/timers.c **** 
  12:Core/Src/timers.c **** 
  13:Core/Src/timers.c **** 
  14:Core/Src/timers.c **** 
  15:Core/Src/timers.c **** /*
  16:Core/Src/timers.c **** #define   TIM3_PRESCALER 16000
  17:Core/Src/timers.c **** #define   TIM3_PERIOD 1000
  18:Core/Src/timers.c **** #define  TIM2_PRESCALER 16
  19:Core/Src/timers.c **** #define  TIM2_PERIOD 10*/
  20:Core/Src/timers.c **** #define   TIM16_PRESCALER 799
  21:Core/Src/timers.c **** #define   TIM16_PERIOD 99
  22:Core/Src/timers.c **** #define   TIM16_PULSE 50
  23:Core/Src/timers.c **** #define  TIM_INTER_PERIOD 9
  24:Core/Src/timers.c **** /*
  25:Core/Src/timers.c **** #define   TIM3_PERIOD 1000
  26:Core/Src/timers.c **** #define  TIM2_PRESCALER 16*/
  27:Core/Src/timers.c **** 
  28:Core/Src/timers.c **** // TIM2 - trigger timertimersr
  29:Core/Src/timers.c **** 
  30:Core/Src/timers.c **** TIM_HandleTypeDef htim2;
  31:Core/Src/timers.c **** TIM_HandleTypeDef htim3;
ARM GAS  /tmp/ccNMEBpy.s 			page 2


  32:Core/Src/timers.c **** TIM_HandleTypeDef htim5;
  33:Core/Src/timers.c **** TIM_HandleTypeDef htim6;
  34:Core/Src/timers.c **** TIM_HandleTypeDef htim16;
  35:Core/Src/timers.c **** TIM_HandleTypeDef htim17;
  36:Core/Src/timers.c **** 
  37:Core/Src/timers.c **** 
  38:Core/Src/timers.c **** static void MX_TIM2_Init(void);
  39:Core/Src/timers.c **** static void MX_TIM5_Init(void);
  40:Core/Src/timers.c **** static void MX_TIM3_Init(void);
  41:Core/Src/timers.c **** static void MX_TIM6_Init(void);
  42:Core/Src/timers.c **** 
  43:Core/Src/timers.c **** static void MX_TIM16_Init(void);
  44:Core/Src/timers.c **** static void MX_TIM17_Init(void);
  45:Core/Src/timers.c **** 
  46:Core/Src/timers.c **** 
  47:Core/Src/timers.c **** 
  48:Core/Src/timers.c **** uint32_t timDiscPeriod = TIM_DISCHARGE_PERIOD;
  49:Core/Src/timers.c **** uint32_t timDiscPulse = TIM_DISCHARGE_PULSE;
  50:Core/Src/timers.c **** uint32_t timTrigPeriod = TIM_TRIGGER_PERIOD;
  51:Core/Src/timers.c **** uint32_t timInterPeriod = TIM_INTER_PERIOD;
  52:Core/Src/timers.c **** uint32_t compareTrigValue = TIM_TRIGGER_COMPARE;
  53:Core/Src/timers.c **** 
  54:Core/Src/timers.c **** uint32_t temp = 0;
  55:Core/Src/timers.c **** //uint32_t timer_set_trigger_period = TIM2_PERIOD;
  56:Core/Src/timers.c **** //uint32_t timer_set_trigger_period = TIM2_PERIOD;
  57:Core/Src/timers.c **** 
  58:Core/Src/timers.c **** void timer_us_delay (uint32_t us)
  59:Core/Src/timers.c **** {
  60:Core/Src/timers.c ****     __HAL_TIM_SET_COUNTER(&htim6,0);
  61:Core/Src/timers.c ****     while ((__HAL_TIM_GET_COUNTER(&htim6))<us);
  62:Core/Src/timers.c **** }
  63:Core/Src/timers.c **** 
  64:Core/Src/timers.c **** void timer_set_trigger_period(uint16_t period){
  65:Core/Src/timers.c ****    // HAL_TIM_Base_Stop(&htim16);
  66:Core/Src/timers.c ****     (&htim2)->Instance->ARR = period;
  67:Core/Src/timers.c ****  //   (&htim16)->Init.Period = period;   
  68:Core/Src/timers.c ****   //  HAL_TIM_Base_Start(&htim16);
  69:Core/Src/timers.c **** }
  70:Core/Src/timers.c **** 
  71:Core/Src/timers.c **** void timer_set_discharge_period(uint16_t period){
  72:Core/Src/timers.c ****    // HAL_TIM_Base_Stop(&htim16);
  73:Core/Src/timers.c ****     (&htim5)->Instance->ARR = period;
  74:Core/Src/timers.c ****  //   (&htim16)->Init.Period = period;   
  75:Core/Src/timers.c ****   //  HAL_TIM_Base_Start(&htim16);
  76:Core/Src/timers.c **** }
  77:Core/Src/timers.c **** 
  78:Core/Src/timers.c **** void timers_trigger_discarge_manually(void)
  79:Core/Src/timers.c **** /*{
  80:Core/Src/timers.c ****     // Ensure TIM3 is not running
  81:Core/Src/timers.c ****     HAL_TIM_PWM_Stop(&htim2, TIM_CHANNEL_3); // Stop PWM generation on TIM3 if it's running
  82:Core/Src/timers.c ****     HAL_TIM_Base_Stop(&htim2);               // Stop the base timer
  83:Core/Src/timers.c **** 
  84:Core/Src/timers.c ****     uint32_t originalValue;
  85:Core/Src/timers.c **** 
  86:Core/Src/timers.c ****     // Assuming TIM2 and Channel 3 are used
  87:Core/Src/timers.c ****     // Save the original value of the CCR register for Channel 3
  88:Core/Src/timers.c ****     originalValue = TIM2->CCR3;
ARM GAS  /tmp/ccNMEBpy.s 			page 3


  89:Core/Src/timers.c **** 
  90:Core/Src/timers.c ****     // Set the CCR register to 0 (either makes the output continuously low or high based on your co
  91:Core/Src/timers.c ****     TIM2->CCR3 = 0;
  92:Core/Src/timers.c **** 
  93:Core/Src/timers.c ****     //HAL_TIM_Base_Start(&htim2);               // Start the base timer
  94:Core/Src/timers.c ****     HAL_TIM_PWM_Start(&htim2, TIM_CHANNEL_3); 
  95:Core/Src/timers.c ****     // Insert a delay
  96:Core/Src/timers.c ****     HAL_Delay(100);  // Delay for 1000 ms or 1 second
  97:Core/Src/timers.c ****     HAL_TIM_PWM_Stop(&htim2, TIM_CHANNEL_3); 
  98:Core/Src/timers.c **** 
  99:Core/Src/timers.c ****     // Restore the original value of the CCR register
 100:Core/Src/timers.c ****     TIM2->CCR3 = originalValue;
 101:Core/Src/timers.c ****     // Start TIM3 in One Pulse Mode
 102:Core/Src/timers.c ****     HAL_TIM_Base_Start(&htim2);  
 103:Core/Src/timers.c ****     HAL_TIM_PWM_Start(&htim2, TIM_CHANNEL_3); 
 104:Core/Src/timers.c ****              // Start the base timer
 105:Core/Src/timers.c ****     //HAL_TIM_PWM_Start(&htim2, TIM_CHANNEL_3); // Start PWM generation on TIM3
 106:Core/Src/timers.c **** }*/
 107:Core/Src/timers.c **** 
 108:Core/Src/timers.c **** {
 109:Core/Src/timers.c ****     // Stop the timer to ensure it doesn't interfere with GPIO manipulation
 110:Core/Src/timers.c ****     HAL_TIM_PWM_Stop(&htim2, TIM_CHANNEL_3); 
 111:Core/Src/timers.c ****     HAL_TIM_Base_Stop(&htim2);
 112:Core/Src/timers.c **** 
 113:Core/Src/timers.c **** 
 114:Core/Src/timers.c ****     // Reconfigure PA2 as a regular output pin
 115:Core/Src/timers.c ****     GPIO_InitTypeDef GPIO_InitStruct = {0};
 116:Core/Src/timers.c ****     GPIO_InitStruct.Pin = GPIO_PIN_2;
 117:Core/Src/timers.c ****     GPIO_InitStruct.Mode = GPIO_MODE_OUTPUT_PP;
 118:Core/Src/timers.c ****     GPIO_InitStruct.Pull = GPIO_NOPULL;
 119:Core/Src/timers.c ****     GPIO_InitStruct.Speed = GPIO_SPEED_FREQ_LOW;
 120:Core/Src/timers.c ****     HAL_GPIO_Init(GPIOA, &GPIO_InitStruct);
 121:Core/Src/timers.c **** 
 122:Core/Src/timers.c ****     // Set the pin high
 123:Core/Src/timers.c ****     HAL_GPIO_WritePin(GPIOA, GPIO_PIN_2, GPIO_PIN_SET);
 124:Core/Src/timers.c **** 
 125:Core/Src/timers.c ****     // Insert a delay if needed
 126:Core/Src/timers.c ****     HAL_Delay(100); // 1000 ms delay
 127:Core/Src/timers.c **** 
 128:Core/Src/timers.c ****     GPIO_InitStruct.Pin = GPIO_PIN_2;
 129:Core/Src/timers.c ****     GPIO_InitStruct.Mode = GPIO_MODE_AF_PP;
 130:Core/Src/timers.c ****     GPIO_InitStruct.Pull = GPIO_NOPULL;
 131:Core/Src/timers.c ****     GPIO_InitStruct.Speed = GPIO_SPEED_FREQ_LOW;
 132:Core/Src/timers.c ****     GPIO_InitStruct.Alternate = GPIO_AF1_TIM2;
 133:Core/Src/timers.c ****     HAL_GPIO_Init(GPIOA, &GPIO_InitStruct);
 134:Core/Src/timers.c **** 
 135:Core/Src/timers.c ****     // Restore the original configuration
 136:Core/Src/timers.c ****     HAL_GPIO_Init(GPIOA, &GPIO_InitStruct);
 137:Core/Src/timers.c **** 
 138:Core/Src/timers.c ****     // Restart the timer
 139:Core/Src/timers.c ****     HAL_TIM_Base_Start(&htim2);  
 140:Core/Src/timers.c ****     HAL_TIM_PWM_Start(&htim2, TIM_CHANNEL_3);
 141:Core/Src/timers.c **** }
 142:Core/Src/timers.c **** 
 143:Core/Src/timers.c **** 
 144:Core/Src/timers.c **** void timers_init_timers(void){
 145:Core/Src/timers.c ****   MX_TIM2_Init(); // discharge
ARM GAS  /tmp/ccNMEBpy.s 			page 4


 146:Core/Src/timers.c ****   MX_TIM5_Init(); // trigger
 147:Core/Src/timers.c ****   MX_TIM3_Init();
 148:Core/Src/timers.c ****   MX_TIM6_Init(); // us delay
 149:Core/Src/timers.c ****   MX_TIM17_Init(); // temperature measuring
 150:Core/Src/timers.c **** 
 151:Core/Src/timers.c ****   if (DEBUG){
 152:Core/Src/timers.c ****       MX_TIM16_Init();
 153:Core/Src/timers.c ****   }
 154:Core/Src/timers.c **** }
 155:Core/Src/timers.c **** void timers_start_timers(void){
 156:Core/Src/timers.c ****   HAL_TIM_Base_Start(&htim2);
 157:Core/Src/timers.c ****   HAL_TIM_Base_Start(&htim3);
 158:Core/Src/timers.c ****   HAL_TIM_Base_Start(&htim5);
 159:Core/Src/timers.c ****   HAL_TIM_Base_Start(&htim6);
 160:Core/Src/timers.c ****   //HAL_TIM_Base_Start(&htim16);
 161:Core/Src/timers.c ****   HAL_TIM_Base_Start_IT(&htim17);
 162:Core/Src/timers.c **** 
 163:Core/Src/timers.c **** }
 164:Core/Src/timers.c **** 
 165:Core/Src/timers.c **** void HAL_TIM_PeriodElapsedCallback(TIM_HandleTypeDef* htim)
 166:Core/Src/timers.c **** {
 167:Core/Src/timers.c ****   temp_convert_temperature();
 168:Core/Src/timers.c **** }
 169:Core/Src/timers.c **** 
 170:Core/Src/timers.c **** 
 171:Core/Src/timers.c **** void timers_start_pwm(void){
 172:Core/Src/timers.c ****   //HAL_TIM_PWM_Start(&htim16, TIM_CHANNEL_1);
 173:Core/Src/timers.c ****   HAL_TIM_PWM_Start(&htim2, TIM_CHANNEL_3);
 174:Core/Src/timers.c ****   if (DEBUG){
 175:Core/Src/timers.c ****       HAL_TIM_PWM_Start(&htim16, TIM_CHANNEL_1);
 176:Core/Src/timers.c ****   }
 177:Core/Src/timers.c ****   //HAL_TIM_PWM_Start(&htim3, TIM_CHANNEL_4);
 178:Core/Src/timers.c **** 
 179:Core/Src/timers.c **** }
 180:Core/Src/timers.c **** 
 181:Core/Src/timers.c **** 
 182:Core/Src/timers.c **** /**
 183:Core/Src/timers.c ****   * @brief TIM2 Initialization Function
 184:Core/Src/timers.c ****   * @param None
 185:Core/Src/timers.c ****   * @retval None
 186:Core/Src/timers.c ****   */
 187:Core/Src/timers.c **** static void MX_TIM5_Init(void)
 188:Core/Src/timers.c **** {
 189:Core/Src/timers.c **** 
 190:Core/Src/timers.c ****   /* USER CODE BEGIN TIM2_Init 0 */
 191:Core/Src/timers.c **** 
 192:Core/Src/timers.c ****   /* USER CODE END TIM2_Init 0 */
 193:Core/Src/timers.c **** 
 194:Core/Src/timers.c ****   TIM_ClockConfigTypeDef sClockSourceConfig = {0};
 195:Core/Src/timers.c ****   TIM_SlaveConfigTypeDef sSlaveConfig = {0};
 196:Core/Src/timers.c ****   TIM_MasterConfigTypeDef sMasterConfig = {0};
 197:Core/Src/timers.c **** 
 198:Core/Src/timers.c ****   /* USER CODE BEGIN TIM2_Init 1 */
 199:Core/Src/timers.c **** 
 200:Core/Src/timers.c ****   /* USER CODE END TIM2_Init 1 */
 201:Core/Src/timers.c ****   htim5.Instance = TIM5;
 202:Core/Src/timers.c ****   htim5.Init.Prescaler = TIM_GLOBAL_PRESCALER;
ARM GAS  /tmp/ccNMEBpy.s 			page 5


 203:Core/Src/timers.c ****   htim5.Init.CounterMode = TIM_COUNTERMODE_UP;
 204:Core/Src/timers.c ****   htim5.Init.Period = timTrigPeriod;
 205:Core/Src/timers.c ****   htim5.Init.ClockDivision = TIM_CLOCKDIVISION_DIV1;
 206:Core/Src/timers.c ****   htim5.Init.AutoReloadPreload = TIM_AUTORELOAD_PRELOAD_DISABLE;
 207:Core/Src/timers.c ****   if (HAL_TIM_Base_Init(&htim5) != HAL_OK)
 208:Core/Src/timers.c ****   {
 209:Core/Src/timers.c ****     Error_Handler();
 210:Core/Src/timers.c ****   }
 211:Core/Src/timers.c ****   sClockSourceConfig.ClockSource = TIM_CLOCKSOURCE_INTERNAL;
 212:Core/Src/timers.c ****   if (HAL_TIM_ConfigClockSource(&htim5, &sClockSourceConfig) != HAL_OK)
 213:Core/Src/timers.c ****   {
 214:Core/Src/timers.c ****     Error_Handler();
 215:Core/Src/timers.c ****   }
 216:Core/Src/timers.c ****   if (HAL_TIM_OnePulse_Init(&htim5, TIM_OPMODE_SINGLE) != HAL_OK)
 217:Core/Src/timers.c ****   {
 218:Core/Src/timers.c ****     Error_Handler();
 219:Core/Src/timers.c ****   }
 220:Core/Src/timers.c ****   sSlaveConfig.SlaveMode = TIM_SLAVEMODE_TRIGGER;
 221:Core/Src/timers.c ****   sSlaveConfig.InputTrigger = TIM_TS_ETRF;
 222:Core/Src/timers.c ****   sSlaveConfig.TriggerPolarity = TIM_TRIGGERPOLARITY_NONINVERTED;
 223:Core/Src/timers.c ****   sSlaveConfig.TriggerPrescaler = TIM_TRIGGERPRESCALER_DIV1;
 224:Core/Src/timers.c ****   sSlaveConfig.TriggerFilter = 0;
 225:Core/Src/timers.c ****   if (HAL_TIM_SlaveConfigSynchro(&htim5, &sSlaveConfig) != HAL_OK)
 226:Core/Src/timers.c ****   {
 227:Core/Src/timers.c ****     Error_Handler();
 228:Core/Src/timers.c ****   }
 229:Core/Src/timers.c ****   sMasterConfig.MasterOutputTrigger = TIM_TRGO_OC1;
 230:Core/Src/timers.c ****   sMasterConfig.MasterSlaveMode = TIM_MASTERSLAVEMODE_DISABLE;
 231:Core/Src/timers.c ****   if (HAL_TIMEx_MasterConfigSynchronization(&htim5, &sMasterConfig) != HAL_OK)
 232:Core/Src/timers.c ****   {
 233:Core/Src/timers.c ****     Error_Handler();
 234:Core/Src/timers.c ****   }
 235:Core/Src/timers.c ****   TIM_OC_InitTypeDef sConfigOC = {0};
 236:Core/Src/timers.c **** 
 237:Core/Src/timers.c ****   sConfigOC.OCMode = TIM_OCMODE_TIMING;
 238:Core/Src/timers.c ****   sConfigOC.Pulse = compareTrigValue;  // Set your compare match value here
 239:Core/Src/timers.c ****   sConfigOC.OCPolarity = TIM_OCPOLARITY_HIGH;
 240:Core/Src/timers.c ****   sConfigOC.OCFastMode = TIM_OCFAST_DISABLE;
 241:Core/Src/timers.c **** 
 242:Core/Src/timers.c ****   if (HAL_TIM_OC_ConfigChannel(&htim5, &sConfigOC, TIM_CHANNEL_1) != HAL_OK)
 243:Core/Src/timers.c ****   {
 244:Core/Src/timers.c ****     Error_Handler();
 245:Core/Src/timers.c ****   }
 246:Core/Src/timers.c ****   
 247:Core/Src/timers.c ****   /* USER CODE BEGIN TIM2_Init 2 */
 248:Core/Src/timers.c **** 
 249:Core/Src/timers.c ****   /* USER CODE END TIM2_Init 2 */
 250:Core/Src/timers.c **** 
 251:Core/Src/timers.c **** }
 252:Core/Src/timers.c **** 
 253:Core/Src/timers.c **** /**
 254:Core/Src/timers.c ****   * @brief TIM3 Initialization Function
 255:Core/Src/timers.c ****   * @param None
 256:Core/Src/timers.c ****   * @retval None
 257:Core/Src/timers.c ****   */
 258:Core/Src/timers.c **** 
 259:Core/Src/timers.c **** static void MX_TIM3_Init(void)
ARM GAS  /tmp/ccNMEBpy.s 			page 6


 260:Core/Src/timers.c **** {
 261:Core/Src/timers.c ****     TIM_SlaveConfigTypeDef sSlaveConfig = {0};
 262:Core/Src/timers.c ****     TIM_MasterConfigTypeDef sMasterConfig = {0};
 263:Core/Src/timers.c **** 
 264:Core/Src/timers.c ****     htim3.Instance = TIM3;
 265:Core/Src/timers.c ****     htim3.Init.Prescaler = TIM_GLOBAL_PRESCALER;
 266:Core/Src/timers.c ****     htim3.Init.CounterMode = TIM_COUNTERMODE_UP;
 267:Core/Src/timers.c ****     htim3.Init.Period = timInterPeriod;  // Set as needed
 268:Core/Src/timers.c ****     htim3.Init.ClockDivision = TIM_CLOCKDIVISION_DIV1;
 269:Core/Src/timers.c ****     htim3.Init.AutoReloadPreload = TIM_AUTORELOAD_PRELOAD_DISABLE;
 270:Core/Src/timers.c ****     if (HAL_TIM_Base_Init(&htim3) != HAL_OK)
 271:Core/Src/timers.c ****     {
 272:Core/Src/timers.c ****         Error_Handler();
 273:Core/Src/timers.c ****     }
 274:Core/Src/timers.c **** 
 275:Core/Src/timers.c ****     // Configuring TIM3 as a slave timer triggered by TIM5
 276:Core/Src/timers.c ****     sSlaveConfig.SlaveMode = TIM_SLAVEMODE_TRIGGER;
 277:Core/Src/timers.c ****     sSlaveConfig.InputTrigger = TIM_TS_ITR4; // ITR4 assumes TIM5 is triggering TIM3
 278:Core/Src/timers.c ****     sSlaveConfig.TriggerPolarity = TIM_TRIGGERPOLARITY_RISING;
 279:Core/Src/timers.c ****     sSlaveConfig.TriggerPrescaler = TIM_TRIGGERPRESCALER_DIV1;
 280:Core/Src/timers.c ****     sSlaveConfig.TriggerFilter = 0;
 281:Core/Src/timers.c ****     if (HAL_TIM_SlaveConfigSynchro(&htim3, &sSlaveConfig) != HAL_OK)
 282:Core/Src/timers.c ****     {
 283:Core/Src/timers.c ****         Error_Handler();
 284:Core/Src/timers.c ****     }
 285:Core/Src/timers.c **** 
 286:Core/Src/timers.c ****     // Configure to generate a TRGO on update event
 287:Core/Src/timers.c ****     sMasterConfig.MasterOutputTrigger = TIM_TRGO_UPDATE;
 288:Core/Src/timers.c ****     sMasterConfig.MasterSlaveMode = TIM_MASTERSLAVEMODE_DISABLE;
 289:Core/Src/timers.c ****     if (HAL_TIMEx_MasterConfigSynchronization(&htim3, &sMasterConfig) != HAL_OK)
 290:Core/Src/timers.c ****     {
 291:Core/Src/timers.c ****         Error_Handler();
 292:Core/Src/timers.c ****     }
 293:Core/Src/timers.c **** 
 294:Core/Src/timers.c ****     // Start TIM3 in One Pulse Mode
 295:Core/Src/timers.c ****     HAL_TIM_OnePulse_Init(&htim3, TIM_OPMODE_SINGLE);
 296:Core/Src/timers.c **** }
 297:Core/Src/timers.c **** 
 298:Core/Src/timers.c **** 
 299:Core/Src/timers.c **** 
 300:Core/Src/timers.c **** /**
 301:Core/Src/timers.c ****   * @brief TIM5 Initialization Function
 302:Core/Src/timers.c ****   * @param None
 303:Core/Src/timers.c ****   * @retval None
 304:Core/Src/timers.c ****   */
 305:Core/Src/timers.c **** static void MX_TIM2_Init(void)
 306:Core/Src/timers.c **** {
 307:Core/Src/timers.c **** 
 308:Core/Src/timers.c ****   /* USER CODE BEGIN TIM5_Init 0 */
 309:Core/Src/timers.c **** 
 310:Core/Src/timers.c ****   /* USER CODE END TIM5_Init 0 */
 311:Core/Src/timers.c **** 
 312:Core/Src/timers.c ****   TIM_ClockConfigTypeDef sClockSourceConfig = {0};
 313:Core/Src/timers.c ****   TIM_SlaveConfigTypeDef sSlaveConfig = {0};
 314:Core/Src/timers.c ****   TIM_MasterConfigTypeDef sMasterConfig = {0};
 315:Core/Src/timers.c ****   TIM_OC_InitTypeDef sConfigOC = {0};
 316:Core/Src/timers.c **** 
ARM GAS  /tmp/ccNMEBpy.s 			page 7


 317:Core/Src/timers.c ****   /* USER CODE BEGIN TIM5_Init 1 */
 318:Core/Src/timers.c **** 
 319:Core/Src/timers.c ****   /* USER CODE END TIM5_Init 1 */
 320:Core/Src/timers.c ****   htim2.Instance = TIM2;
 321:Core/Src/timers.c ****   htim2.Init.Prescaler = TIM_GLOBAL_PRESCALER;
 322:Core/Src/timers.c ****   htim2.Init.CounterMode = TIM_COUNTERMODE_UP;
 323:Core/Src/timers.c ****   htim2.Init.Period = timDiscPeriod;
 324:Core/Src/timers.c ****   htim2.Init.ClockDivision = TIM_CLOCKDIVISION_DIV1;
 325:Core/Src/timers.c ****   htim2.Init.AutoReloadPreload = TIM_AUTORELOAD_PRELOAD_DISABLE;
 326:Core/Src/timers.c ****   if (HAL_TIM_Base_Init(&htim2) != HAL_OK)
 327:Core/Src/timers.c ****   {
 328:Core/Src/timers.c ****     Error_Handler();
 329:Core/Src/timers.c ****   }
 330:Core/Src/timers.c ****   sClockSourceConfig.ClockSource = TIM_CLOCKSOURCE_INTERNAL;
 331:Core/Src/timers.c ****   if (HAL_TIM_ConfigClockSource(&htim2, &sClockSourceConfig) != HAL_OK)
 332:Core/Src/timers.c ****   {
 333:Core/Src/timers.c ****     Error_Handler();
 334:Core/Src/timers.c ****   }
 335:Core/Src/timers.c ****   if (HAL_TIM_PWM_Init(&htim2) != HAL_OK)
 336:Core/Src/timers.c ****   {
 337:Core/Src/timers.c ****     Error_Handler();
 338:Core/Src/timers.c ****   }
 339:Core/Src/timers.c ****   if (HAL_TIM_OnePulse_Init(&htim2, TIM_OPMODE_SINGLE) != HAL_OK)
 340:Core/Src/timers.c ****   {
 341:Core/Src/timers.c ****     Error_Handler();
 342:Core/Src/timers.c ****   }
 343:Core/Src/timers.c ****   sSlaveConfig.SlaveMode = TIM_SLAVEMODE_TRIGGER;
 344:Core/Src/timers.c ****   sSlaveConfig.InputTrigger = TIM_TS_ITR2;
 345:Core/Src/timers.c ****   if (HAL_TIM_SlaveConfigSynchro(&htim2, &sSlaveConfig) != HAL_OK)
 346:Core/Src/timers.c ****   {
 347:Core/Src/timers.c ****     Error_Handler();
 348:Core/Src/timers.c ****   }
 349:Core/Src/timers.c ****   sMasterConfig.MasterOutputTrigger = TIM_TRGO_UPDATE;
 350:Core/Src/timers.c ****   sMasterConfig.MasterSlaveMode = TIM_MASTERSLAVEMODE_DISABLE;
 351:Core/Src/timers.c ****   if (HAL_TIMEx_MasterConfigSynchronization(&htim2, &sMasterConfig) != HAL_OK)
 352:Core/Src/timers.c ****   {
 353:Core/Src/timers.c ****     Error_Handler();
 354:Core/Src/timers.c ****   }
 355:Core/Src/timers.c ****   sConfigOC.OCMode = TIM_OCMODE_PWM1;
 356:Core/Src/timers.c ****   sConfigOC.Pulse = timDiscPulse;
 357:Core/Src/timers.c ****   sConfigOC.OCPolarity = TIM_OCPOLARITY_LOW;
 358:Core/Src/timers.c ****   sConfigOC.OCFastMode = TIM_OCFAST_DISABLE;
 359:Core/Src/timers.c ****   if (HAL_TIM_PWM_ConfigChannel(&htim2, &sConfigOC, TIM_CHANNEL_3) != HAL_OK)
 360:Core/Src/timers.c ****   {
 361:Core/Src/timers.c ****     Error_Handler();
 362:Core/Src/timers.c ****   }
 363:Core/Src/timers.c ****   /* USER CODE BEGIN TIM5_Init 2 */
 364:Core/Src/timers.c **** 
 365:Core/Src/timers.c ****   /* USER CODE END TIM5_Init 2 */
 366:Core/Src/timers.c ****   HAL_TIM_MspPostInit(&htim2);
 367:Core/Src/timers.c **** 
 368:Core/Src/timers.c **** }
 369:Core/Src/timers.c **** 
 370:Core/Src/timers.c **** /**
 371:Core/Src/timers.c ****   * @brief TIM16 Initialization Function
 372:Core/Src/timers.c ****   * @param None
 373:Core/Src/timers.c ****   * @retval None
ARM GAS  /tmp/ccNMEBpy.s 			page 8


 374:Core/Src/timers.c ****   */
 375:Core/Src/timers.c **** static void MX_TIM16_Init(void)
 376:Core/Src/timers.c **** {
 377:Core/Src/timers.c **** 
 378:Core/Src/timers.c ****   /* USER CODE BEGIN TIM16_Init 0 */
 379:Core/Src/timers.c **** 
 380:Core/Src/timers.c ****   /* USER CODE END TIM16_Init 0 */
 381:Core/Src/timers.c **** 
 382:Core/Src/timers.c ****   TIM_OC_InitTypeDef sConfigOC = {0};
 383:Core/Src/timers.c ****   TIM_BreakDeadTimeConfigTypeDef sBreakDeadTimeConfig = {0};
 384:Core/Src/timers.c **** 
 385:Core/Src/timers.c ****   /* USER CODE BEGIN TIM16_Init 1 */
 386:Core/Src/timers.c **** 
 387:Core/Src/timers.c ****   /* USER CODE END TIM16_Init 1 */
 388:Core/Src/timers.c ****   htim16.Instance = TIM16;
 389:Core/Src/timers.c ****   htim16.Init.Prescaler = TIM16_PRESCALER;
 390:Core/Src/timers.c ****   htim16.Init.CounterMode = TIM_COUNTERMODE_UP;
 391:Core/Src/timers.c ****   htim16.Init.Period = TIM16_PERIOD;
 392:Core/Src/timers.c ****   htim16.Init.ClockDivision = TIM_CLOCKDIVISION_DIV1;
 393:Core/Src/timers.c ****   htim16.Init.RepetitionCounter = 0;
 394:Core/Src/timers.c ****   htim16.Init.AutoReloadPreload = TIM_AUTORELOAD_PRELOAD_DISABLE;
 395:Core/Src/timers.c ****   if (HAL_TIM_Base_Init(&htim16) != HAL_OK)
 396:Core/Src/timers.c ****   {
 397:Core/Src/timers.c ****     Error_Handler();
 398:Core/Src/timers.c ****   }
 399:Core/Src/timers.c ****   if (HAL_TIM_PWM_Init(&htim16) != HAL_OK)
 400:Core/Src/timers.c ****   {
 401:Core/Src/timers.c ****     Error_Handler();
 402:Core/Src/timers.c ****   }
 403:Core/Src/timers.c ****   sConfigOC.OCMode = TIM_OCMODE_PWM1;
 404:Core/Src/timers.c ****   sConfigOC.Pulse = TIM16_PULSE;
 405:Core/Src/timers.c ****   sConfigOC.OCPolarity = TIM_OCPOLARITY_LOW;
 406:Core/Src/timers.c ****   sConfigOC.OCNPolarity = TIM_OCNPOLARITY_HIGH;
 407:Core/Src/timers.c ****   sConfigOC.OCFastMode = TIM_OCFAST_DISABLE;
 408:Core/Src/timers.c ****   sConfigOC.OCIdleState = TIM_OCIDLESTATE_RESET;
 409:Core/Src/timers.c ****   sConfigOC.OCNIdleState = TIM_OCNIDLESTATE_RESET;
 410:Core/Src/timers.c ****   if (HAL_TIM_PWM_ConfigChannel(&htim16, &sConfigOC, TIM_CHANNEL_1) != HAL_OK)
 411:Core/Src/timers.c ****   {
 412:Core/Src/timers.c ****     Error_Handler();
 413:Core/Src/timers.c ****   }
 414:Core/Src/timers.c ****   sBreakDeadTimeConfig.OffStateRunMode = TIM_OSSR_DISABLE;
 415:Core/Src/timers.c ****   sBreakDeadTimeConfig.OffStateIDLEMode = TIM_OSSI_DISABLE;
 416:Core/Src/timers.c ****   sBreakDeadTimeConfig.LockLevel = TIM_LOCKLEVEL_OFF;
 417:Core/Src/timers.c ****   sBreakDeadTimeConfig.DeadTime = 0;
 418:Core/Src/timers.c ****   sBreakDeadTimeConfig.BreakState = TIM_BREAK_DISABLE;
 419:Core/Src/timers.c ****   sBreakDeadTimeConfig.BreakPolarity = TIM_BREAKPOLARITY_HIGH;
 420:Core/Src/timers.c ****   sBreakDeadTimeConfig.BreakFilter = 0;
 421:Core/Src/timers.c ****   sBreakDeadTimeConfig.AutomaticOutput = TIM_AUTOMATICOUTPUT_DISABLE;
 422:Core/Src/timers.c ****   if (HAL_TIMEx_ConfigBreakDeadTime(&htim16, &sBreakDeadTimeConfig) != HAL_OK)
 423:Core/Src/timers.c ****   {
 424:Core/Src/timers.c ****     Error_Handler();
 425:Core/Src/timers.c ****   }
 426:Core/Src/timers.c ****   /* USER CODE BEGIN TIM16_Init 2 */
 427:Core/Src/timers.c **** 
 428:Core/Src/timers.c ****   /* USER CODE END TIM16_Init 2 */
 429:Core/Src/timers.c ****   HAL_TIM_MspPostInit(&htim16);
 430:Core/Src/timers.c **** 
ARM GAS  /tmp/ccNMEBpy.s 			page 9


 431:Core/Src/timers.c **** }
 432:Core/Src/timers.c **** 
 433:Core/Src/timers.c **** static void MX_TIM17_Init(void)
 434:Core/Src/timers.c **** {
  28              		.loc 1 434 1 view -0
  29              		.cfi_startproc
  30              		@ args = 0, pretend = 0, frame = 0
  31              		@ frame_needed = 0, uses_anonymous_args = 0
  32 0000 08B5     		push	{r3, lr}
  33              		.cfi_def_cfa_offset 8
  34              		.cfi_offset 3, -8
  35              		.cfi_offset 14, -4
 435:Core/Src/timers.c **** 
 436:Core/Src/timers.c ****   /* USER CODE BEGIN TIM17_Init 0 */
 437:Core/Src/timers.c **** 
 438:Core/Src/timers.c ****   /* USER CODE END TIM17_Init 0 */
 439:Core/Src/timers.c **** 
 440:Core/Src/timers.c ****   /* USER CODE BEGIN TIM17_Init 1 */
 441:Core/Src/timers.c **** 
 442:Core/Src/timers.c ****   /* USER CODE ETIM_HandleTypeDef htim17;
 443:Core/Src/timers.c ****    * ND TIM17_Init 1 */
 444:Core/Src/timers.c ****   htim17.Instance = TIM17;
  36              		.loc 1 444 3 view .LVU1
  37              		.loc 1 444 19 is_stmt 0 view .LVU2
  38 0002 0A48     		ldr	r0, .L5
  39 0004 0A4B     		ldr	r3, .L5+4
  40 0006 0360     		str	r3, [r0]
 445:Core/Src/timers.c ****   htim17.Init.Prescaler = TIM_TEMP_PRESCALER;
  41              		.loc 1 445 3 is_stmt 1 view .LVU3
  42              		.loc 1 445 25 is_stmt 0 view .LVU4
  43 0008 49F63F43 		movw	r3, #39999
  44 000c 4360     		str	r3, [r0, #4]
 446:Core/Src/timers.c ****   htim17.Init.CounterMode = TIM_COUNTERMODE_UP;
  45              		.loc 1 446 3 is_stmt 1 view .LVU5
  46              		.loc 1 446 27 is_stmt 0 view .LVU6
  47 000e 0023     		movs	r3, #0
  48 0010 8360     		str	r3, [r0, #8]
 447:Core/Src/timers.c ****   htim17.Init.Period = TIM_TEMP_PERIOD;
  49              		.loc 1 447 3 is_stmt 1 view .LVU7
  50              		.loc 1 447 22 is_stmt 0 view .LVU8
  51 0012 44F62062 		movw	r2, #20000
  52 0016 C260     		str	r2, [r0, #12]
 448:Core/Src/timers.c ****   htim17.Init.ClockDivision = TIM_CLOCKDIVISION_DIV1;
  53              		.loc 1 448 3 is_stmt 1 view .LVU9
  54              		.loc 1 448 29 is_stmt 0 view .LVU10
  55 0018 0361     		str	r3, [r0, #16]
 449:Core/Src/timers.c ****   htim17.Init.RepetitionCounter = 0;
  56              		.loc 1 449 3 is_stmt 1 view .LVU11
  57              		.loc 1 449 33 is_stmt 0 view .LVU12
  58 001a 4361     		str	r3, [r0, #20]
 450:Core/Src/timers.c ****   htim17.Init.AutoReloadPreload = TIM_AUTORELOAD_PRELOAD_DISABLE;
  59              		.loc 1 450 3 is_stmt 1 view .LVU13
  60              		.loc 1 450 33 is_stmt 0 view .LVU14
  61 001c 8361     		str	r3, [r0, #24]
 451:Core/Src/timers.c ****   if (HAL_TIM_Base_Init(&htim17) != HAL_OK)
  62              		.loc 1 451 3 is_stmt 1 view .LVU15
  63              		.loc 1 451 7 is_stmt 0 view .LVU16
ARM GAS  /tmp/ccNMEBpy.s 			page 10


  64 001e FFF7FEFF 		bl	HAL_TIM_Base_Init
  65              	.LVL0:
  66              		.loc 1 451 6 view .LVU17
  67 0022 00B9     		cbnz	r0, .L4
  68              	.L1:
 452:Core/Src/timers.c ****   {
 453:Core/Src/timers.c ****     Error_Handler();
 454:Core/Src/timers.c ****   }
 455:Core/Src/timers.c ****   /* USER CODE BEGIN TIM17_Init 2 */
 456:Core/Src/timers.c **** 
 457:Core/Src/timers.c ****   /* USER CODE END TIM17_Init 2 */
 458:Core/Src/timers.c **** 
 459:Core/Src/timers.c **** }
  69              		.loc 1 459 1 view .LVU18
  70 0024 08BD     		pop	{r3, pc}
  71              	.L4:
 453:Core/Src/timers.c ****   }
  72              		.loc 1 453 5 is_stmt 1 view .LVU19
  73 0026 FFF7FEFF 		bl	Error_Handler
  74              	.LVL1:
  75              		.loc 1 459 1 is_stmt 0 view .LVU20
  76 002a FBE7     		b	.L1
  77              	.L6:
  78              		.align	2
  79              	.L5:
  80 002c 00000000 		.word	htim17
  81 0030 00480140 		.word	1073825792
  82              		.cfi_endproc
  83              	.LFE341:
  85              		.section	.text.MX_TIM3_Init,"ax",%progbits
  86              		.align	1
  87              		.syntax unified
  88              		.thumb
  89              		.thumb_func
  90              		.fpu fpv4-sp-d16
  92              	MX_TIM3_Init:
  93              	.LFB338:
 260:Core/Src/timers.c ****     TIM_SlaveConfigTypeDef sSlaveConfig = {0};
  94              		.loc 1 260 1 is_stmt 1 view -0
  95              		.cfi_startproc
  96              		@ args = 0, pretend = 0, frame = 32
  97              		@ frame_needed = 0, uses_anonymous_args = 0
  98 0000 00B5     		push	{lr}
  99              		.cfi_def_cfa_offset 4
 100              		.cfi_offset 14, -4
 101 0002 89B0     		sub	sp, sp, #36
 102              		.cfi_def_cfa_offset 40
 261:Core/Src/timers.c ****     TIM_MasterConfigTypeDef sMasterConfig = {0};
 103              		.loc 1 261 5 view .LVU22
 261:Core/Src/timers.c ****     TIM_MasterConfigTypeDef sMasterConfig = {0};
 104              		.loc 1 261 28 is_stmt 0 view .LVU23
 105 0004 0023     		movs	r3, #0
 106 0006 0393     		str	r3, [sp, #12]
 107 0008 0493     		str	r3, [sp, #16]
 108 000a 0593     		str	r3, [sp, #20]
 109 000c 0693     		str	r3, [sp, #24]
 110 000e 0793     		str	r3, [sp, #28]
ARM GAS  /tmp/ccNMEBpy.s 			page 11


 262:Core/Src/timers.c **** 
 111              		.loc 1 262 5 is_stmt 1 view .LVU24
 262:Core/Src/timers.c **** 
 112              		.loc 1 262 29 is_stmt 0 view .LVU25
 113 0010 0093     		str	r3, [sp]
 114 0012 0193     		str	r3, [sp, #4]
 115 0014 0293     		str	r3, [sp, #8]
 264:Core/Src/timers.c ****     htim3.Init.Prescaler = TIM_GLOBAL_PRESCALER;
 116              		.loc 1 264 5 is_stmt 1 view .LVU26
 264:Core/Src/timers.c ****     htim3.Init.Prescaler = TIM_GLOBAL_PRESCALER;
 117              		.loc 1 264 20 is_stmt 0 view .LVU27
 118 0016 1A48     		ldr	r0, .L15
 119 0018 1A4A     		ldr	r2, .L15+4
 120 001a 0260     		str	r2, [r0]
 265:Core/Src/timers.c ****     htim3.Init.CounterMode = TIM_COUNTERMODE_UP;
 121              		.loc 1 265 5 is_stmt 1 view .LVU28
 265:Core/Src/timers.c ****     htim3.Init.CounterMode = TIM_COUNTERMODE_UP;
 122              		.loc 1 265 26 is_stmt 0 view .LVU29
 123 001c 0122     		movs	r2, #1
 124 001e 4260     		str	r2, [r0, #4]
 266:Core/Src/timers.c ****     htim3.Init.Period = timInterPeriod;  // Set as needed
 125              		.loc 1 266 5 is_stmt 1 view .LVU30
 266:Core/Src/timers.c ****     htim3.Init.Period = timInterPeriod;  // Set as needed
 126              		.loc 1 266 28 is_stmt 0 view .LVU31
 127 0020 8360     		str	r3, [r0, #8]
 267:Core/Src/timers.c ****     htim3.Init.ClockDivision = TIM_CLOCKDIVISION_DIV1;
 128              		.loc 1 267 5 is_stmt 1 view .LVU32
 267:Core/Src/timers.c ****     htim3.Init.ClockDivision = TIM_CLOCKDIVISION_DIV1;
 129              		.loc 1 267 23 is_stmt 0 view .LVU33
 130 0022 194A     		ldr	r2, .L15+8
 131 0024 1268     		ldr	r2, [r2]
 132 0026 C260     		str	r2, [r0, #12]
 268:Core/Src/timers.c ****     htim3.Init.AutoReloadPreload = TIM_AUTORELOAD_PRELOAD_DISABLE;
 133              		.loc 1 268 5 is_stmt 1 view .LVU34
 268:Core/Src/timers.c ****     htim3.Init.AutoReloadPreload = TIM_AUTORELOAD_PRELOAD_DISABLE;
 134              		.loc 1 268 30 is_stmt 0 view .LVU35
 135 0028 0361     		str	r3, [r0, #16]
 269:Core/Src/timers.c ****     if (HAL_TIM_Base_Init(&htim3) != HAL_OK)
 136              		.loc 1 269 5 is_stmt 1 view .LVU36
 269:Core/Src/timers.c ****     if (HAL_TIM_Base_Init(&htim3) != HAL_OK)
 137              		.loc 1 269 34 is_stmt 0 view .LVU37
 138 002a 8361     		str	r3, [r0, #24]
 270:Core/Src/timers.c ****     {
 139              		.loc 1 270 5 is_stmt 1 view .LVU38
 270:Core/Src/timers.c ****     {
 140              		.loc 1 270 9 is_stmt 0 view .LVU39
 141 002c FFF7FEFF 		bl	HAL_TIM_Base_Init
 142              	.LVL2:
 270:Core/Src/timers.c ****     {
 143              		.loc 1 270 8 view .LVU40
 144 0030 E8B9     		cbnz	r0, .L12
 145              	.L8:
 276:Core/Src/timers.c ****     sSlaveConfig.InputTrigger = TIM_TS_ITR4; // ITR4 assumes TIM5 is triggering TIM3
 146              		.loc 1 276 5 is_stmt 1 view .LVU41
 276:Core/Src/timers.c ****     sSlaveConfig.InputTrigger = TIM_TS_ITR4; // ITR4 assumes TIM5 is triggering TIM3
 147              		.loc 1 276 28 is_stmt 0 view .LVU42
 148 0032 0623     		movs	r3, #6
ARM GAS  /tmp/ccNMEBpy.s 			page 12


 149 0034 0393     		str	r3, [sp, #12]
 277:Core/Src/timers.c ****     sSlaveConfig.TriggerPolarity = TIM_TRIGGERPOLARITY_RISING;
 150              		.loc 1 277 5 is_stmt 1 view .LVU43
 277:Core/Src/timers.c ****     sSlaveConfig.TriggerPolarity = TIM_TRIGGERPOLARITY_RISING;
 151              		.loc 1 277 31 is_stmt 0 view .LVU44
 152 0036 4FF48013 		mov	r3, #1048576
 153 003a 0493     		str	r3, [sp, #16]
 278:Core/Src/timers.c ****     sSlaveConfig.TriggerPrescaler = TIM_TRIGGERPRESCALER_DIV1;
 154              		.loc 1 278 5 is_stmt 1 view .LVU45
 278:Core/Src/timers.c ****     sSlaveConfig.TriggerPrescaler = TIM_TRIGGERPRESCALER_DIV1;
 155              		.loc 1 278 34 is_stmt 0 view .LVU46
 156 003c 0023     		movs	r3, #0
 157 003e 0593     		str	r3, [sp, #20]
 279:Core/Src/timers.c ****     sSlaveConfig.TriggerFilter = 0;
 158              		.loc 1 279 5 is_stmt 1 view .LVU47
 279:Core/Src/timers.c ****     sSlaveConfig.TriggerFilter = 0;
 159              		.loc 1 279 35 is_stmt 0 view .LVU48
 160 0040 0693     		str	r3, [sp, #24]
 280:Core/Src/timers.c ****     if (HAL_TIM_SlaveConfigSynchro(&htim3, &sSlaveConfig) != HAL_OK)
 161              		.loc 1 280 5 is_stmt 1 view .LVU49
 280:Core/Src/timers.c ****     if (HAL_TIM_SlaveConfigSynchro(&htim3, &sSlaveConfig) != HAL_OK)
 162              		.loc 1 280 32 is_stmt 0 view .LVU50
 163 0042 0793     		str	r3, [sp, #28]
 281:Core/Src/timers.c ****     {
 164              		.loc 1 281 5 is_stmt 1 view .LVU51
 281:Core/Src/timers.c ****     {
 165              		.loc 1 281 9 is_stmt 0 view .LVU52
 166 0044 03A9     		add	r1, sp, #12
 167 0046 0E48     		ldr	r0, .L15
 168 0048 FFF7FEFF 		bl	HAL_TIM_SlaveConfigSynchro
 169              	.LVL3:
 281:Core/Src/timers.c ****     {
 170              		.loc 1 281 8 view .LVU53
 171 004c 90B9     		cbnz	r0, .L13
 172              	.L9:
 287:Core/Src/timers.c ****     sMasterConfig.MasterSlaveMode = TIM_MASTERSLAVEMODE_DISABLE;
 173              		.loc 1 287 5 is_stmt 1 view .LVU54
 287:Core/Src/timers.c ****     sMasterConfig.MasterSlaveMode = TIM_MASTERSLAVEMODE_DISABLE;
 174              		.loc 1 287 39 is_stmt 0 view .LVU55
 175 004e 2023     		movs	r3, #32
 176 0050 0093     		str	r3, [sp]
 288:Core/Src/timers.c ****     if (HAL_TIMEx_MasterConfigSynchronization(&htim3, &sMasterConfig) != HAL_OK)
 177              		.loc 1 288 5 is_stmt 1 view .LVU56
 288:Core/Src/timers.c ****     if (HAL_TIMEx_MasterConfigSynchronization(&htim3, &sMasterConfig) != HAL_OK)
 178              		.loc 1 288 35 is_stmt 0 view .LVU57
 179 0052 0023     		movs	r3, #0
 180 0054 0293     		str	r3, [sp, #8]
 289:Core/Src/timers.c ****     {
 181              		.loc 1 289 5 is_stmt 1 view .LVU58
 289:Core/Src/timers.c ****     {
 182              		.loc 1 289 9 is_stmt 0 view .LVU59
 183 0056 6946     		mov	r1, sp
 184 0058 0948     		ldr	r0, .L15
 185 005a FFF7FEFF 		bl	HAL_TIMEx_MasterConfigSynchronization
 186              	.LVL4:
 289:Core/Src/timers.c ****     {
 187              		.loc 1 289 8 view .LVU60
ARM GAS  /tmp/ccNMEBpy.s 			page 13


 188 005e 60B9     		cbnz	r0, .L14
 189              	.L10:
 295:Core/Src/timers.c **** }
 190              		.loc 1 295 5 is_stmt 1 view .LVU61
 191 0060 0821     		movs	r1, #8
 192 0062 0748     		ldr	r0, .L15
 193 0064 FFF7FEFF 		bl	HAL_TIM_OnePulse_Init
 194              	.LVL5:
 296:Core/Src/timers.c **** 
 195              		.loc 1 296 1 is_stmt 0 view .LVU62
 196 0068 09B0     		add	sp, sp, #36
 197              		.cfi_remember_state
 198              		.cfi_def_cfa_offset 4
 199              		@ sp needed
 200 006a 5DF804FB 		ldr	pc, [sp], #4
 201              	.L12:
 202              		.cfi_restore_state
 272:Core/Src/timers.c ****     }
 203              		.loc 1 272 9 is_stmt 1 view .LVU63
 204 006e FFF7FEFF 		bl	Error_Handler
 205              	.LVL6:
 206 0072 DEE7     		b	.L8
 207              	.L13:
 283:Core/Src/timers.c ****     }
 208              		.loc 1 283 9 view .LVU64
 209 0074 FFF7FEFF 		bl	Error_Handler
 210              	.LVL7:
 211 0078 E9E7     		b	.L9
 212              	.L14:
 291:Core/Src/timers.c ****     }
 213              		.loc 1 291 9 view .LVU65
 214 007a FFF7FEFF 		bl	Error_Handler
 215              	.LVL8:
 216 007e EFE7     		b	.L10
 217              	.L16:
 218              		.align	2
 219              	.L15:
 220 0080 00000000 		.word	htim3
 221 0084 00040040 		.word	1073742848
 222 0088 00000000 		.word	.LANCHOR0
 223              		.cfi_endproc
 224              	.LFE338:
 226              		.section	.text.MX_TIM6_Init,"ax",%progbits
 227              		.align	1
 228              		.syntax unified
 229              		.thumb
 230              		.thumb_func
 231              		.fpu fpv4-sp-d16
 233              	MX_TIM6_Init:
 234              	.LFB342:
 460:Core/Src/timers.c **** 
 461:Core/Src/timers.c **** 
 462:Core/Src/timers.c **** 
 463:Core/Src/timers.c **** static void MX_TIM6_Init(void)
 464:Core/Src/timers.c **** {
 235              		.loc 1 464 1 view -0
 236              		.cfi_startproc
ARM GAS  /tmp/ccNMEBpy.s 			page 14


 237              		@ args = 0, pretend = 0, frame = 16
 238              		@ frame_needed = 0, uses_anonymous_args = 0
 239 0000 00B5     		push	{lr}
 240              		.cfi_def_cfa_offset 4
 241              		.cfi_offset 14, -4
 242 0002 85B0     		sub	sp, sp, #20
 243              		.cfi_def_cfa_offset 24
 465:Core/Src/timers.c **** 
 466:Core/Src/timers.c ****   /* USER CODE BEGIN TIM6_Init 0 */
 467:Core/Src/timers.c **** 
 468:Core/Src/timers.c ****   /* USER CODE END TIM6_Init 0 */
 469:Core/Src/timers.c **** 
 470:Core/Src/timers.c ****   TIM_MasterConfigTypeDef sMasterConfig = {0};
 244              		.loc 1 470 3 view .LVU67
 245              		.loc 1 470 27 is_stmt 0 view .LVU68
 246 0004 0023     		movs	r3, #0
 247 0006 0193     		str	r3, [sp, #4]
 248 0008 0293     		str	r3, [sp, #8]
 249 000a 0393     		str	r3, [sp, #12]
 471:Core/Src/timers.c **** 
 472:Core/Src/timers.c ****   /* USER CODE BEGIN TIM6_Init 1 */
 473:Core/Src/timers.c **** 
 474:Core/Src/timers.c ****   /* USER CODE END TIM6_Init 1 */
 475:Core/Src/timers.c ****   htim6.Instance = TIM6;
 250              		.loc 1 475 3 is_stmt 1 view .LVU69
 251              		.loc 1 475 18 is_stmt 0 view .LVU70
 252 000c 0E48     		ldr	r0, .L23
 253 000e 0F4A     		ldr	r2, .L23+4
 254 0010 0260     		str	r2, [r0]
 476:Core/Src/timers.c ****   htim6.Init.Prescaler = 79;
 255              		.loc 1 476 3 is_stmt 1 view .LVU71
 256              		.loc 1 476 24 is_stmt 0 view .LVU72
 257 0012 4F22     		movs	r2, #79
 258 0014 4260     		str	r2, [r0, #4]
 477:Core/Src/timers.c ****   htim6.Init.CounterMode = TIM_COUNTERMODE_UP;
 259              		.loc 1 477 3 is_stmt 1 view .LVU73
 260              		.loc 1 477 26 is_stmt 0 view .LVU74
 261 0016 8360     		str	r3, [r0, #8]
 478:Core/Src/timers.c ****   htim6.Init.Period = 65535;
 262              		.loc 1 478 3 is_stmt 1 view .LVU75
 263              		.loc 1 478 21 is_stmt 0 view .LVU76
 264 0018 4FF6FF72 		movw	r2, #65535
 265 001c C260     		str	r2, [r0, #12]
 479:Core/Src/timers.c ****   htim6.Init.AutoReloadPreload = TIM_AUTORELOAD_PRELOAD_DISABLE;
 266              		.loc 1 479 3 is_stmt 1 view .LVU77
 267              		.loc 1 479 32 is_stmt 0 view .LVU78
 268 001e 8361     		str	r3, [r0, #24]
 480:Core/Src/timers.c ****   if (HAL_TIM_Base_Init(&htim6) != HAL_OK)
 269              		.loc 1 480 3 is_stmt 1 view .LVU79
 270              		.loc 1 480 7 is_stmt 0 view .LVU80
 271 0020 FFF7FEFF 		bl	HAL_TIM_Base_Init
 272              	.LVL9:
 273              		.loc 1 480 6 view .LVU81
 274 0024 50B9     		cbnz	r0, .L21
 275              	.L18:
 481:Core/Src/timers.c ****   {
 482:Core/Src/timers.c ****     Error_Handler();
ARM GAS  /tmp/ccNMEBpy.s 			page 15


 483:Core/Src/timers.c ****   }
 484:Core/Src/timers.c ****   sMasterConfig.MasterOutputTrigger = TIM_TRGO_RESET;
 276              		.loc 1 484 3 is_stmt 1 view .LVU82
 277              		.loc 1 484 37 is_stmt 0 view .LVU83
 278 0026 0023     		movs	r3, #0
 279 0028 0193     		str	r3, [sp, #4]
 485:Core/Src/timers.c ****   sMasterConfig.MasterSlaveMode = TIM_MASTERSLAVEMODE_DISABLE;
 280              		.loc 1 485 3 is_stmt 1 view .LVU84
 281              		.loc 1 485 33 is_stmt 0 view .LVU85
 282 002a 0393     		str	r3, [sp, #12]
 486:Core/Src/timers.c ****   if (HAL_TIMEx_MasterConfigSynchronization(&htim6, &sMasterConfig) != HAL_OK)
 283              		.loc 1 486 3 is_stmt 1 view .LVU86
 284              		.loc 1 486 7 is_stmt 0 view .LVU87
 285 002c 01A9     		add	r1, sp, #4
 286 002e 0648     		ldr	r0, .L23
 287 0030 FFF7FEFF 		bl	HAL_TIMEx_MasterConfigSynchronization
 288              	.LVL10:
 289              		.loc 1 486 6 view .LVU88
 290 0034 28B9     		cbnz	r0, .L22
 291              	.L17:
 487:Core/Src/timers.c ****   {
 488:Core/Src/timers.c ****     Error_Handler();
 489:Core/Src/timers.c ****   }
 490:Core/Src/timers.c ****   /* USER CODE BEGIN TIM6_Init 2 */
 491:Core/Src/timers.c **** 
 492:Core/Src/timers.c ****   /* USER CODE END TIM6_Init 2 */
 493:Core/Src/timers.c **** 
 494:Core/Src/timers.c **** }...
 292              		.loc 1 494 1 view .LVU89
 293 0036 05B0     		add	sp, sp, #20
 294              		.cfi_remember_state
 295              		.cfi_def_cfa_offset 4
 296              		@ sp needed
 297 0038 5DF804FB 		ldr	pc, [sp], #4
 298              	.L21:
 299              		.cfi_restore_state
 482:Core/Src/timers.c ****     Error_Handler();
 300              		.loc 1 482 5 is_stmt 1 view .LVU90
 301 003c FFF7FEFF 		bl	Error_Handler
 302              	.LVL11:
 303 0040 F1E7     		b	.L18
 304              	.L22:
 488:Core/Src/timers.c ****     Error_Handler();
 305              		.loc 1 488 5 view .LVU91
 306 0042 FFF7FEFF 		bl	Error_Handler
 307              	.LVL12:
 308              		.loc 1 494 1 is_stmt 0 view .LVU92
 309 0046 F6E7     		b	.L17
 310              	.L24:
 311              		.align	2
 312              	.L23:
 313 0048 00000000 		.word	htim6
 314 004c 00100040 		.word	1073745920
 315              		.cfi_endproc
 316              	.LFE342:
 318              		.section	.text.MX_TIM2_Init,"ax",%progbits
 319              		.align	1
ARM GAS  /tmp/ccNMEBpy.s 			page 16


 320              		.syntax unified
 321              		.thumb
 322              		.thumb_func
 323              		.fpu fpv4-sp-d16
 325              	MX_TIM2_Init:
 326              	.LFB339:
 306:Core/Src/timers.c **** {
 327              		.loc 1 306 1 is_stmt 1 view -0
 328              		.cfi_startproc
 329              		@ args = 0, pretend = 0, frame = 80
 330              		@ frame_needed = 0, uses_anonymous_args = 0
 331 0000 00B5     		push	{lr}
 332              		.cfi_def_cfa_offset 4
 333              		.cfi_offset 14, -4
 334 0002 95B0     		sub	sp, sp, #84
 335              		.cfi_def_cfa_offset 88
 312:Core/Src/timers.c ****   TIM_ClockConfigTypeDef sClockSourceConfig = {0};
 336              		.loc 1 312 3 view .LVU94
 312:Core/Src/timers.c ****   TIM_ClockConfigTypeDef sClockSourceConfig = {0};
 337              		.loc 1 312 26 is_stmt 0 view .LVU95
 338 0004 0023     		movs	r3, #0
 339 0006 1093     		str	r3, [sp, #64]
 340 0008 1193     		str	r3, [sp, #68]
 341 000a 1293     		str	r3, [sp, #72]
 342 000c 1393     		str	r3, [sp, #76]
 313:Core/Src/timers.c ****   TIM_SlaveConfigTypeDef sSlaveConfig = {0};
 343              		.loc 1 313 3 is_stmt 1 view .LVU96
 313:Core/Src/timers.c ****   TIM_SlaveConfigTypeDef sSlaveConfig = {0};
 344              		.loc 1 313 26 is_stmt 0 view .LVU97
 345 000e 0B93     		str	r3, [sp, #44]
 346 0010 0C93     		str	r3, [sp, #48]
 347 0012 0D93     		str	r3, [sp, #52]
 348 0014 0E93     		str	r3, [sp, #56]
 349 0016 0F93     		str	r3, [sp, #60]
 314:Core/Src/timers.c ****   TIM_MasterConfigTypeDef sMasterConfig = {0};
 350              		.loc 1 314 3 is_stmt 1 view .LVU98
 314:Core/Src/timers.c ****   TIM_MasterConfigTypeDef sMasterConfig = {0};
 351              		.loc 1 314 27 is_stmt 0 view .LVU99
 352 0018 0893     		str	r3, [sp, #32]
 353 001a 0993     		str	r3, [sp, #36]
 354 001c 0A93     		str	r3, [sp, #40]
 315:Core/Src/timers.c ****   TIM_OC_InitTypeDef sConfigOC = {0};
 355              		.loc 1 315 3 is_stmt 1 view .LVU100
 315:Core/Src/timers.c ****   TIM_OC_InitTypeDef sConfigOC = {0};
 356              		.loc 1 315 22 is_stmt 0 view .LVU101
 357 001e 0193     		str	r3, [sp, #4]
 358 0020 0293     		str	r3, [sp, #8]
 359 0022 0393     		str	r3, [sp, #12]
 360 0024 0493     		str	r3, [sp, #16]
 361 0026 0593     		str	r3, [sp, #20]
 362 0028 0693     		str	r3, [sp, #24]
 363 002a 0793     		str	r3, [sp, #28]
 320:Core/Src/timers.c ****   htim2.Instance = TIM2;
 364              		.loc 1 320 3 is_stmt 1 view .LVU102
 320:Core/Src/timers.c ****   htim2.Instance = TIM2;
 365              		.loc 1 320 18 is_stmt 0 view .LVU103
 366 002c 2F48     		ldr	r0, .L41
ARM GAS  /tmp/ccNMEBpy.s 			page 17


 367 002e 4FF08042 		mov	r2, #1073741824
 368 0032 0260     		str	r2, [r0]
 321:Core/Src/timers.c ****   htim2.Init.Prescaler = TIM_GLOBAL_PRESCALER;
 369              		.loc 1 321 3 is_stmt 1 view .LVU104
 321:Core/Src/timers.c ****   htim2.Init.Prescaler = TIM_GLOBAL_PRESCALER;
 370              		.loc 1 321 24 is_stmt 0 view .LVU105
 371 0034 0122     		movs	r2, #1
 372 0036 4260     		str	r2, [r0, #4]
 322:Core/Src/timers.c ****   htim2.Init.CounterMode = TIM_COUNTERMODE_UP;
 373              		.loc 1 322 3 is_stmt 1 view .LVU106
 322:Core/Src/timers.c ****   htim2.Init.CounterMode = TIM_COUNTERMODE_UP;
 374              		.loc 1 322 26 is_stmt 0 view .LVU107
 375 0038 8360     		str	r3, [r0, #8]
 323:Core/Src/timers.c ****   htim2.Init.Period = timDiscPeriod;
 376              		.loc 1 323 3 is_stmt 1 view .LVU108
 323:Core/Src/timers.c ****   htim2.Init.Period = timDiscPeriod;
 377              		.loc 1 323 21 is_stmt 0 view .LVU109
 378 003a 2D4A     		ldr	r2, .L41+4
 379 003c 1268     		ldr	r2, [r2]
 380 003e C260     		str	r2, [r0, #12]
 324:Core/Src/timers.c ****   htim2.Init.ClockDivision = TIM_CLOCKDIVISION_DIV1;
 381              		.loc 1 324 3 is_stmt 1 view .LVU110
 324:Core/Src/timers.c ****   htim2.Init.ClockDivision = TIM_CLOCKDIVISION_DIV1;
 382              		.loc 1 324 28 is_stmt 0 view .LVU111
 383 0040 0361     		str	r3, [r0, #16]
 325:Core/Src/timers.c ****   htim2.Init.AutoReloadPreload = TIM_AUTORELOAD_PRELOAD_DISABLE;
 384              		.loc 1 325 3 is_stmt 1 view .LVU112
 325:Core/Src/timers.c ****   htim2.Init.AutoReloadPreload = TIM_AUTORELOAD_PRELOAD_DISABLE;
 385              		.loc 1 325 32 is_stmt 0 view .LVU113
 386 0042 8361     		str	r3, [r0, #24]
 326:Core/Src/timers.c ****   if (HAL_TIM_Base_Init(&htim2) != HAL_OK)
 387              		.loc 1 326 3 is_stmt 1 view .LVU114
 326:Core/Src/timers.c ****   if (HAL_TIM_Base_Init(&htim2) != HAL_OK)
 388              		.loc 1 326 7 is_stmt 0 view .LVU115
 389 0044 FFF7FEFF 		bl	HAL_TIM_Base_Init
 390              	.LVL13:
 326:Core/Src/timers.c ****   if (HAL_TIM_Base_Init(&htim2) != HAL_OK)
 391              		.loc 1 326 6 view .LVU116
 392 0048 0028     		cmp	r0, #0
 393 004a 3AD1     		bne	.L34
 394              	.L26:
 330:Core/Src/timers.c ****   sClockSourceConfig.ClockSource = TIM_CLOCKSOURCE_INTERNAL;
 395              		.loc 1 330 3 is_stmt 1 view .LVU117
 330:Core/Src/timers.c ****   sClockSourceConfig.ClockSource = TIM_CLOCKSOURCE_INTERNAL;
 396              		.loc 1 330 34 is_stmt 0 view .LVU118
 397 004c 4FF48053 		mov	r3, #4096
 398 0050 1093     		str	r3, [sp, #64]
 331:Core/Src/timers.c ****   if (HAL_TIM_ConfigClockSource(&htim2, &sClockSourceConfig) != HAL_OK)
 399              		.loc 1 331 3 is_stmt 1 view .LVU119
 331:Core/Src/timers.c ****   if (HAL_TIM_ConfigClockSource(&htim2, &sClockSourceConfig) != HAL_OK)
 400              		.loc 1 331 7 is_stmt 0 view .LVU120
 401 0052 10A9     		add	r1, sp, #64
 402 0054 2548     		ldr	r0, .L41
 403 0056 FFF7FEFF 		bl	HAL_TIM_ConfigClockSource
 404              	.LVL14:
 331:Core/Src/timers.c ****   if (HAL_TIM_ConfigClockSource(&htim2, &sClockSourceConfig) != HAL_OK)
 405              		.loc 1 331 6 view .LVU121
ARM GAS  /tmp/ccNMEBpy.s 			page 18


 406 005a 0028     		cmp	r0, #0
 407 005c 34D1     		bne	.L35
 408              	.L27:
 335:Core/Src/timers.c ****   if (HAL_TIM_PWM_Init(&htim2) != HAL_OK)
 409              		.loc 1 335 3 is_stmt 1 view .LVU122
 335:Core/Src/timers.c ****   if (HAL_TIM_PWM_Init(&htim2) != HAL_OK)
 410              		.loc 1 335 7 is_stmt 0 view .LVU123
 411 005e 2348     		ldr	r0, .L41
 412 0060 FFF7FEFF 		bl	HAL_TIM_PWM_Init
 413              	.LVL15:
 335:Core/Src/timers.c ****   if (HAL_TIM_PWM_Init(&htim2) != HAL_OK)
 414              		.loc 1 335 6 view .LVU124
 415 0064 0028     		cmp	r0, #0
 416 0066 32D1     		bne	.L36
 417              	.L28:
 339:Core/Src/timers.c ****   if (HAL_TIM_OnePulse_Init(&htim2, TIM_OPMODE_SINGLE) != HAL_OK)
 418              		.loc 1 339 3 is_stmt 1 view .LVU125
 339:Core/Src/timers.c ****   if (HAL_TIM_OnePulse_Init(&htim2, TIM_OPMODE_SINGLE) != HAL_OK)
 419              		.loc 1 339 7 is_stmt 0 view .LVU126
 420 0068 0821     		movs	r1, #8
 421 006a 2048     		ldr	r0, .L41
 422 006c FFF7FEFF 		bl	HAL_TIM_OnePulse_Init
 423              	.LVL16:
 339:Core/Src/timers.c ****   if (HAL_TIM_OnePulse_Init(&htim2, TIM_OPMODE_SINGLE) != HAL_OK)
 424              		.loc 1 339 6 view .LVU127
 425 0070 0028     		cmp	r0, #0
 426 0072 2FD1     		bne	.L37
 427              	.L29:
 343:Core/Src/timers.c ****   sSlaveConfig.SlaveMode = TIM_SLAVEMODE_TRIGGER;
 428              		.loc 1 343 3 is_stmt 1 view .LVU128
 343:Core/Src/timers.c ****   sSlaveConfig.SlaveMode = TIM_SLAVEMODE_TRIGGER;
 429              		.loc 1 343 26 is_stmt 0 view .LVU129
 430 0074 0623     		movs	r3, #6
 431 0076 0B93     		str	r3, [sp, #44]
 344:Core/Src/timers.c ****   sSlaveConfig.InputTrigger = TIM_TS_ITR2;
 432              		.loc 1 344 3 is_stmt 1 view .LVU130
 344:Core/Src/timers.c ****   sSlaveConfig.InputTrigger = TIM_TS_ITR2;
 433              		.loc 1 344 29 is_stmt 0 view .LVU131
 434 0078 2023     		movs	r3, #32
 435 007a 0C93     		str	r3, [sp, #48]
 345:Core/Src/timers.c ****   if (HAL_TIM_SlaveConfigSynchro(&htim2, &sSlaveConfig) != HAL_OK)
 436              		.loc 1 345 3 is_stmt 1 view .LVU132
 345:Core/Src/timers.c ****   if (HAL_TIM_SlaveConfigSynchro(&htim2, &sSlaveConfig) != HAL_OK)
 437              		.loc 1 345 7 is_stmt 0 view .LVU133
 438 007c 0BA9     		add	r1, sp, #44
 439 007e 1B48     		ldr	r0, .L41
 440 0080 FFF7FEFF 		bl	HAL_TIM_SlaveConfigSynchro
 441              	.LVL17:
 345:Core/Src/timers.c ****   if (HAL_TIM_SlaveConfigSynchro(&htim2, &sSlaveConfig) != HAL_OK)
 442              		.loc 1 345 6 view .LVU134
 443 0084 48BB     		cbnz	r0, .L38
 444              	.L30:
 349:Core/Src/timers.c ****   sMasterConfig.MasterOutputTrigger = TIM_TRGO_UPDATE;
 445              		.loc 1 349 3 is_stmt 1 view .LVU135
 349:Core/Src/timers.c ****   sMasterConfig.MasterOutputTrigger = TIM_TRGO_UPDATE;
 446              		.loc 1 349 37 is_stmt 0 view .LVU136
 447 0086 2023     		movs	r3, #32
ARM GAS  /tmp/ccNMEBpy.s 			page 19


 448 0088 0893     		str	r3, [sp, #32]
 350:Core/Src/timers.c ****   sMasterConfig.MasterSlaveMode = TIM_MASTERSLAVEMODE_DISABLE;
 449              		.loc 1 350 3 is_stmt 1 view .LVU137
 350:Core/Src/timers.c ****   sMasterConfig.MasterSlaveMode = TIM_MASTERSLAVEMODE_DISABLE;
 450              		.loc 1 350 33 is_stmt 0 view .LVU138
 451 008a 0023     		movs	r3, #0
 452 008c 0A93     		str	r3, [sp, #40]
 351:Core/Src/timers.c ****   if (HAL_TIMEx_MasterConfigSynchronization(&htim2, &sMasterConfig) != HAL_OK)
 453              		.loc 1 351 3 is_stmt 1 view .LVU139
 351:Core/Src/timers.c ****   if (HAL_TIMEx_MasterConfigSynchronization(&htim2, &sMasterConfig) != HAL_OK)
 454              		.loc 1 351 7 is_stmt 0 view .LVU140
 455 008e 08A9     		add	r1, sp, #32
 456 0090 1648     		ldr	r0, .L41
 457 0092 FFF7FEFF 		bl	HAL_TIMEx_MasterConfigSynchronization
 458              	.LVL18:
 351:Core/Src/timers.c ****   if (HAL_TIMEx_MasterConfigSynchronization(&htim2, &sMasterConfig) != HAL_OK)
 459              		.loc 1 351 6 view .LVU141
 460 0096 18BB     		cbnz	r0, .L39
 461              	.L31:
 355:Core/Src/timers.c ****   sConfigOC.OCMode = TIM_OCMODE_PWM1;
 462              		.loc 1 355 3 is_stmt 1 view .LVU142
 355:Core/Src/timers.c ****   sConfigOC.OCMode = TIM_OCMODE_PWM1;
 463              		.loc 1 355 20 is_stmt 0 view .LVU143
 464 0098 6023     		movs	r3, #96
 465 009a 0193     		str	r3, [sp, #4]
 356:Core/Src/timers.c ****   sConfigOC.Pulse = timDiscPulse;
 466              		.loc 1 356 3 is_stmt 1 view .LVU144
 356:Core/Src/timers.c ****   sConfigOC.Pulse = timDiscPulse;
 467              		.loc 1 356 19 is_stmt 0 view .LVU145
 468 009c 154B     		ldr	r3, .L41+8
 469 009e 1B68     		ldr	r3, [r3]
 470 00a0 0293     		str	r3, [sp, #8]
 357:Core/Src/timers.c ****   sConfigOC.OCPolarity = TIM_OCPOLARITY_LOW;
 471              		.loc 1 357 3 is_stmt 1 view .LVU146
 357:Core/Src/timers.c ****   sConfigOC.OCPolarity = TIM_OCPOLARITY_LOW;
 472              		.loc 1 357 24 is_stmt 0 view .LVU147
 473 00a2 0223     		movs	r3, #2
 474 00a4 0393     		str	r3, [sp, #12]
 358:Core/Src/timers.c ****   sConfigOC.OCFastMode = TIM_OCFAST_DISABLE;
 475              		.loc 1 358 3 is_stmt 1 view .LVU148
 358:Core/Src/timers.c ****   sConfigOC.OCFastMode = TIM_OCFAST_DISABLE;
 476              		.loc 1 358 24 is_stmt 0 view .LVU149
 477 00a6 0023     		movs	r3, #0
 478 00a8 0593     		str	r3, [sp, #20]
 359:Core/Src/timers.c ****   if (HAL_TIM_PWM_ConfigChannel(&htim2, &sConfigOC, TIM_CHANNEL_3) != HAL_OK)
 479              		.loc 1 359 3 is_stmt 1 view .LVU150
 359:Core/Src/timers.c ****   if (HAL_TIM_PWM_ConfigChannel(&htim2, &sConfigOC, TIM_CHANNEL_3) != HAL_OK)
 480              		.loc 1 359 7 is_stmt 0 view .LVU151
 481 00aa 0822     		movs	r2, #8
 482 00ac 01A9     		add	r1, sp, #4
 483 00ae 0F48     		ldr	r0, .L41
 484 00b0 FFF7FEFF 		bl	HAL_TIM_PWM_ConfigChannel
 485              	.LVL19:
 359:Core/Src/timers.c ****   if (HAL_TIM_PWM_ConfigChannel(&htim2, &sConfigOC, TIM_CHANNEL_3) != HAL_OK)
 486              		.loc 1 359 6 view .LVU152
 487 00b4 B8B9     		cbnz	r0, .L40
 488              	.L32:
ARM GAS  /tmp/ccNMEBpy.s 			page 20


 366:Core/Src/timers.c ****   HAL_TIM_MspPostInit(&htim2);
 489              		.loc 1 366 3 is_stmt 1 view .LVU153
 490 00b6 0D48     		ldr	r0, .L41
 491 00b8 FFF7FEFF 		bl	HAL_TIM_MspPostInit
 492              	.LVL20:
 368:Core/Src/timers.c **** }
 493              		.loc 1 368 1 is_stmt 0 view .LVU154
 494 00bc 15B0     		add	sp, sp, #84
 495              		.cfi_remember_state
 496              		.cfi_def_cfa_offset 4
 497              		@ sp needed
 498 00be 5DF804FB 		ldr	pc, [sp], #4
 499              	.L34:
 500              		.cfi_restore_state
 328:Core/Src/timers.c ****     Error_Handler();
 501              		.loc 1 328 5 is_stmt 1 view .LVU155
 502 00c2 FFF7FEFF 		bl	Error_Handler
 503              	.LVL21:
 504 00c6 C1E7     		b	.L26
 505              	.L35:
 333:Core/Src/timers.c ****     Error_Handler();
 506              		.loc 1 333 5 view .LVU156
 507 00c8 FFF7FEFF 		bl	Error_Handler
 508              	.LVL22:
 509 00cc C7E7     		b	.L27
 510              	.L36:
 337:Core/Src/timers.c ****     Error_Handler();
 511              		.loc 1 337 5 view .LVU157
 512 00ce FFF7FEFF 		bl	Error_Handler
 513              	.LVL23:
 514 00d2 C9E7     		b	.L28
 515              	.L37:
 341:Core/Src/timers.c ****     Error_Handler();
 516              		.loc 1 341 5 view .LVU158
 517 00d4 FFF7FEFF 		bl	Error_Handler
 518              	.LVL24:
 519 00d8 CCE7     		b	.L29
 520              	.L38:
 347:Core/Src/timers.c ****     Error_Handler();
 521              		.loc 1 347 5 view .LVU159
 522 00da FFF7FEFF 		bl	Error_Handler
 523              	.LVL25:
 524 00de D2E7     		b	.L30
 525              	.L39:
 353:Core/Src/timers.c ****     Error_Handler();
 526              		.loc 1 353 5 view .LVU160
 527 00e0 FFF7FEFF 		bl	Error_Handler
 528              	.LVL26:
 529 00e4 D8E7     		b	.L31
 530              	.L40:
 361:Core/Src/timers.c ****     Error_Handler();
 531              		.loc 1 361 5 view .LVU161
 532 00e6 FFF7FEFF 		bl	Error_Handler
 533              	.LVL27:
 534 00ea E4E7     		b	.L32
 535              	.L42:
 536              		.align	2
ARM GAS  /tmp/ccNMEBpy.s 			page 21


 537              	.L41:
 538 00ec 00000000 		.word	htim2
 539 00f0 00000000 		.word	.LANCHOR1
 540 00f4 00000000 		.word	.LANCHOR2
 541              		.cfi_endproc
 542              	.LFE339:
 544              		.section	.text.MX_TIM5_Init,"ax",%progbits
 545              		.align	1
 546              		.syntax unified
 547              		.thumb
 548              		.thumb_func
 549              		.fpu fpv4-sp-d16
 551              	MX_TIM5_Init:
 552              	.LFB337:
 188:Core/Src/timers.c **** {
 553              		.loc 1 188 1 view -0
 554              		.cfi_startproc
 555              		@ args = 0, pretend = 0, frame = 80
 556              		@ frame_needed = 0, uses_anonymous_args = 0
 557 0000 00B5     		push	{lr}
 558              		.cfi_def_cfa_offset 4
 559              		.cfi_offset 14, -4
 560 0002 95B0     		sub	sp, sp, #84
 561              		.cfi_def_cfa_offset 88
 194:Core/Src/timers.c ****   TIM_ClockConfigTypeDef sClockSourceConfig = {0};
 562              		.loc 1 194 3 view .LVU163
 194:Core/Src/timers.c ****   TIM_ClockConfigTypeDef sClockSourceConfig = {0};
 563              		.loc 1 194 26 is_stmt 0 view .LVU164
 564 0004 0023     		movs	r3, #0
 565 0006 1093     		str	r3, [sp, #64]
 566 0008 1193     		str	r3, [sp, #68]
 567 000a 1293     		str	r3, [sp, #72]
 568 000c 1393     		str	r3, [sp, #76]
 195:Core/Src/timers.c ****   TIM_SlaveConfigTypeDef sSlaveConfig = {0};
 569              		.loc 1 195 3 is_stmt 1 view .LVU165
 195:Core/Src/timers.c ****   TIM_SlaveConfigTypeDef sSlaveConfig = {0};
 570              		.loc 1 195 26 is_stmt 0 view .LVU166
 571 000e 0B93     		str	r3, [sp, #44]
 572 0010 0C93     		str	r3, [sp, #48]
 573 0012 0D93     		str	r3, [sp, #52]
 574 0014 0E93     		str	r3, [sp, #56]
 575 0016 0F93     		str	r3, [sp, #60]
 196:Core/Src/timers.c ****   TIM_MasterConfigTypeDef sMasterConfig = {0};
 576              		.loc 1 196 3 is_stmt 1 view .LVU167
 196:Core/Src/timers.c ****   TIM_MasterConfigTypeDef sMasterConfig = {0};
 577              		.loc 1 196 27 is_stmt 0 view .LVU168
 578 0018 0893     		str	r3, [sp, #32]
 579 001a 0993     		str	r3, [sp, #36]
 580 001c 0A93     		str	r3, [sp, #40]
 201:Core/Src/timers.c ****   htim5.Instance = TIM5;
 581              		.loc 1 201 3 is_stmt 1 view .LVU169
 201:Core/Src/timers.c ****   htim5.Instance = TIM5;
 582              		.loc 1 201 18 is_stmt 0 view .LVU170
 583 001e 2C48     		ldr	r0, .L57
 584 0020 2C4A     		ldr	r2, .L57+4
 585 0022 0260     		str	r2, [r0]
 202:Core/Src/timers.c ****   htim5.Init.Prescaler = TIM_GLOBAL_PRESCALER;
ARM GAS  /tmp/ccNMEBpy.s 			page 22


 586              		.loc 1 202 3 is_stmt 1 view .LVU171
 202:Core/Src/timers.c ****   htim5.Init.Prescaler = TIM_GLOBAL_PRESCALER;
 587              		.loc 1 202 24 is_stmt 0 view .LVU172
 588 0024 0122     		movs	r2, #1
 589 0026 4260     		str	r2, [r0, #4]
 203:Core/Src/timers.c ****   htim5.Init.CounterMode = TIM_COUNTERMODE_UP;
 590              		.loc 1 203 3 is_stmt 1 view .LVU173
 203:Core/Src/timers.c ****   htim5.Init.CounterMode = TIM_COUNTERMODE_UP;
 591              		.loc 1 203 26 is_stmt 0 view .LVU174
 592 0028 8360     		str	r3, [r0, #8]
 204:Core/Src/timers.c ****   htim5.Init.Period = timTrigPeriod;
 593              		.loc 1 204 3 is_stmt 1 view .LVU175
 204:Core/Src/timers.c ****   htim5.Init.Period = timTrigPeriod;
 594              		.loc 1 204 21 is_stmt 0 view .LVU176
 595 002a 2B4A     		ldr	r2, .L57+8
 596 002c 1268     		ldr	r2, [r2]
 597 002e C260     		str	r2, [r0, #12]
 205:Core/Src/timers.c ****   htim5.Init.ClockDivision = TIM_CLOCKDIVISION_DIV1;
 598              		.loc 1 205 3 is_stmt 1 view .LVU177
 205:Core/Src/timers.c ****   htim5.Init.ClockDivision = TIM_CLOCKDIVISION_DIV1;
 599              		.loc 1 205 28 is_stmt 0 view .LVU178
 600 0030 0361     		str	r3, [r0, #16]
 206:Core/Src/timers.c ****   htim5.Init.AutoReloadPreload = TIM_AUTORELOAD_PRELOAD_DISABLE;
 601              		.loc 1 206 3 is_stmt 1 view .LVU179
 206:Core/Src/timers.c ****   htim5.Init.AutoReloadPreload = TIM_AUTORELOAD_PRELOAD_DISABLE;
 602              		.loc 1 206 32 is_stmt 0 view .LVU180
 603 0032 8361     		str	r3, [r0, #24]
 207:Core/Src/timers.c ****   if (HAL_TIM_Base_Init(&htim5) != HAL_OK)
 604              		.loc 1 207 3 is_stmt 1 view .LVU181
 207:Core/Src/timers.c ****   if (HAL_TIM_Base_Init(&htim5) != HAL_OK)
 605              		.loc 1 207 7 is_stmt 0 view .LVU182
 606 0034 FFF7FEFF 		bl	HAL_TIM_Base_Init
 607              	.LVL28:
 207:Core/Src/timers.c ****   if (HAL_TIM_Base_Init(&htim5) != HAL_OK)
 608              		.loc 1 207 6 view .LVU183
 609 0038 0028     		cmp	r0, #0
 610 003a 36D1     		bne	.L51
 611              	.L44:
 211:Core/Src/timers.c ****   sClockSourceConfig.ClockSource = TIM_CLOCKSOURCE_INTERNAL;
 612              		.loc 1 211 3 is_stmt 1 view .LVU184
 211:Core/Src/timers.c ****   sClockSourceConfig.ClockSource = TIM_CLOCKSOURCE_INTERNAL;
 613              		.loc 1 211 34 is_stmt 0 view .LVU185
 614 003c 4FF48053 		mov	r3, #4096
 615 0040 1093     		str	r3, [sp, #64]
 212:Core/Src/timers.c ****   if (HAL_TIM_ConfigClockSource(&htim5, &sClockSourceConfig) != HAL_OK)
 616              		.loc 1 212 3 is_stmt 1 view .LVU186
 212:Core/Src/timers.c ****   if (HAL_TIM_ConfigClockSource(&htim5, &sClockSourceConfig) != HAL_OK)
 617              		.loc 1 212 7 is_stmt 0 view .LVU187
 618 0042 10A9     		add	r1, sp, #64
 619 0044 2248     		ldr	r0, .L57
 620 0046 FFF7FEFF 		bl	HAL_TIM_ConfigClockSource
 621              	.LVL29:
 212:Core/Src/timers.c ****   if (HAL_TIM_ConfigClockSource(&htim5, &sClockSourceConfig) != HAL_OK)
 622              		.loc 1 212 6 view .LVU188
 623 004a 0028     		cmp	r0, #0
 624 004c 30D1     		bne	.L52
 625              	.L45:
ARM GAS  /tmp/ccNMEBpy.s 			page 23


 216:Core/Src/timers.c ****   if (HAL_TIM_OnePulse_Init(&htim5, TIM_OPMODE_SINGLE) != HAL_OK)
 626              		.loc 1 216 3 is_stmt 1 view .LVU189
 216:Core/Src/timers.c ****   if (HAL_TIM_OnePulse_Init(&htim5, TIM_OPMODE_SINGLE) != HAL_OK)
 627              		.loc 1 216 7 is_stmt 0 view .LVU190
 628 004e 0821     		movs	r1, #8
 629 0050 1F48     		ldr	r0, .L57
 630 0052 FFF7FEFF 		bl	HAL_TIM_OnePulse_Init
 631              	.LVL30:
 216:Core/Src/timers.c ****   if (HAL_TIM_OnePulse_Init(&htim5, TIM_OPMODE_SINGLE) != HAL_OK)
 632              		.loc 1 216 6 view .LVU191
 633 0056 0028     		cmp	r0, #0
 634 0058 2DD1     		bne	.L53
 635              	.L46:
 220:Core/Src/timers.c ****   sSlaveConfig.SlaveMode = TIM_SLAVEMODE_TRIGGER;
 636              		.loc 1 220 3 is_stmt 1 view .LVU192
 220:Core/Src/timers.c ****   sSlaveConfig.SlaveMode = TIM_SLAVEMODE_TRIGGER;
 637              		.loc 1 220 26 is_stmt 0 view .LVU193
 638 005a 0623     		movs	r3, #6
 639 005c 0B93     		str	r3, [sp, #44]
 221:Core/Src/timers.c ****   sSlaveConfig.InputTrigger = TIM_TS_ETRF;
 640              		.loc 1 221 3 is_stmt 1 view .LVU194
 221:Core/Src/timers.c ****   sSlaveConfig.InputTrigger = TIM_TS_ETRF;
 641              		.loc 1 221 29 is_stmt 0 view .LVU195
 642 005e 7023     		movs	r3, #112
 643 0060 0C93     		str	r3, [sp, #48]
 222:Core/Src/timers.c ****   sSlaveConfig.TriggerPolarity = TIM_TRIGGERPOLARITY_NONINVERTED;
 644              		.loc 1 222 3 is_stmt 1 view .LVU196
 222:Core/Src/timers.c ****   sSlaveConfig.TriggerPolarity = TIM_TRIGGERPOLARITY_NONINVERTED;
 645              		.loc 1 222 32 is_stmt 0 view .LVU197
 646 0062 0023     		movs	r3, #0
 647 0064 0D93     		str	r3, [sp, #52]
 223:Core/Src/timers.c ****   sSlaveConfig.TriggerPrescaler = TIM_TRIGGERPRESCALER_DIV1;
 648              		.loc 1 223 3 is_stmt 1 view .LVU198
 223:Core/Src/timers.c ****   sSlaveConfig.TriggerPrescaler = TIM_TRIGGERPRESCALER_DIV1;
 649              		.loc 1 223 33 is_stmt 0 view .LVU199
 650 0066 0E93     		str	r3, [sp, #56]
 224:Core/Src/timers.c ****   sSlaveConfig.TriggerFilter = 0;
 651              		.loc 1 224 3 is_stmt 1 view .LVU200
 224:Core/Src/timers.c ****   sSlaveConfig.TriggerFilter = 0;
 652              		.loc 1 224 30 is_stmt 0 view .LVU201
 653 0068 0F93     		str	r3, [sp, #60]
 225:Core/Src/timers.c ****   if (HAL_TIM_SlaveConfigSynchro(&htim5, &sSlaveConfig) != HAL_OK)
 654              		.loc 1 225 3 is_stmt 1 view .LVU202
 225:Core/Src/timers.c ****   if (HAL_TIM_SlaveConfigSynchro(&htim5, &sSlaveConfig) != HAL_OK)
 655              		.loc 1 225 7 is_stmt 0 view .LVU203
 656 006a 0BA9     		add	r1, sp, #44
 657 006c 1848     		ldr	r0, .L57
 658 006e FFF7FEFF 		bl	HAL_TIM_SlaveConfigSynchro
 659              	.LVL31:
 225:Core/Src/timers.c ****   if (HAL_TIM_SlaveConfigSynchro(&htim5, &sSlaveConfig) != HAL_OK)
 660              		.loc 1 225 6 view .LVU204
 661 0072 18BB     		cbnz	r0, .L54
 662              	.L47:
 229:Core/Src/timers.c ****   sMasterConfig.MasterOutputTrigger = TIM_TRGO_OC1;
 663              		.loc 1 229 3 is_stmt 1 view .LVU205
 229:Core/Src/timers.c ****   sMasterConfig.MasterOutputTrigger = TIM_TRGO_OC1;
 664              		.loc 1 229 37 is_stmt 0 view .LVU206
ARM GAS  /tmp/ccNMEBpy.s 			page 24


 665 0074 3023     		movs	r3, #48
 666 0076 0893     		str	r3, [sp, #32]
 230:Core/Src/timers.c ****   sMasterConfig.MasterSlaveMode = TIM_MASTERSLAVEMODE_DISABLE;
 667              		.loc 1 230 3 is_stmt 1 view .LVU207
 230:Core/Src/timers.c ****   sMasterConfig.MasterSlaveMode = TIM_MASTERSLAVEMODE_DISABLE;
 668              		.loc 1 230 33 is_stmt 0 view .LVU208
 669 0078 0023     		movs	r3, #0
 670 007a 0A93     		str	r3, [sp, #40]
 231:Core/Src/timers.c ****   if (HAL_TIMEx_MasterConfigSynchronization(&htim5, &sMasterConfig) != HAL_OK)
 671              		.loc 1 231 3 is_stmt 1 view .LVU209
 231:Core/Src/timers.c ****   if (HAL_TIMEx_MasterConfigSynchronization(&htim5, &sMasterConfig) != HAL_OK)
 672              		.loc 1 231 7 is_stmt 0 view .LVU210
 673 007c 08A9     		add	r1, sp, #32
 674 007e 1448     		ldr	r0, .L57
 675 0080 FFF7FEFF 		bl	HAL_TIMEx_MasterConfigSynchronization
 676              	.LVL32:
 231:Core/Src/timers.c ****   if (HAL_TIMEx_MasterConfigSynchronization(&htim5, &sMasterConfig) != HAL_OK)
 677              		.loc 1 231 6 view .LVU211
 678 0084 E8B9     		cbnz	r0, .L55
 679              	.L48:
 235:Core/Src/timers.c ****   TIM_OC_InitTypeDef sConfigOC = {0};
 680              		.loc 1 235 3 is_stmt 1 view .LVU212
 235:Core/Src/timers.c ****   TIM_OC_InitTypeDef sConfigOC = {0};
 681              		.loc 1 235 22 is_stmt 0 view .LVU213
 682 0086 0022     		movs	r2, #0
 683 0088 0492     		str	r2, [sp, #16]
 684 008a 0692     		str	r2, [sp, #24]
 685 008c 0792     		str	r2, [sp, #28]
 237:Core/Src/timers.c ****   sConfigOC.OCMode = TIM_OCMODE_TIMING;
 686              		.loc 1 237 3 is_stmt 1 view .LVU214
 237:Core/Src/timers.c ****   sConfigOC.OCMode = TIM_OCMODE_TIMING;
 687              		.loc 1 237 20 is_stmt 0 view .LVU215
 688 008e 0192     		str	r2, [sp, #4]
 238:Core/Src/timers.c ****   sConfigOC.Pulse = compareTrigValue;  // Set your compare match value here
 689              		.loc 1 238 3 is_stmt 1 view .LVU216
 238:Core/Src/timers.c ****   sConfigOC.Pulse = compareTrigValue;  // Set your compare match value here
 690              		.loc 1 238 19 is_stmt 0 view .LVU217
 691 0090 124B     		ldr	r3, .L57+12
 692 0092 1B68     		ldr	r3, [r3]
 693 0094 0293     		str	r3, [sp, #8]
 239:Core/Src/timers.c ****   sConfigOC.OCPolarity = TIM_OCPOLARITY_HIGH;
 694              		.loc 1 239 3 is_stmt 1 view .LVU218
 239:Core/Src/timers.c ****   sConfigOC.OCPolarity = TIM_OCPOLARITY_HIGH;
 695              		.loc 1 239 24 is_stmt 0 view .LVU219
 696 0096 0392     		str	r2, [sp, #12]
 240:Core/Src/timers.c ****   sConfigOC.OCFastMode = TIM_OCFAST_DISABLE;
 697              		.loc 1 240 3 is_stmt 1 view .LVU220
 240:Core/Src/timers.c ****   sConfigOC.OCFastMode = TIM_OCFAST_DISABLE;
 698              		.loc 1 240 24 is_stmt 0 view .LVU221
 699 0098 0592     		str	r2, [sp, #20]
 242:Core/Src/timers.c ****   if (HAL_TIM_OC_ConfigChannel(&htim5, &sConfigOC, TIM_CHANNEL_1) != HAL_OK)
 700              		.loc 1 242 3 is_stmt 1 view .LVU222
 242:Core/Src/timers.c ****   if (HAL_TIM_OC_ConfigChannel(&htim5, &sConfigOC, TIM_CHANNEL_1) != HAL_OK)
 701              		.loc 1 242 7 is_stmt 0 view .LVU223
 702 009a 01A9     		add	r1, sp, #4
 703 009c 0C48     		ldr	r0, .L57
 704 009e FFF7FEFF 		bl	HAL_TIM_OC_ConfigChannel
ARM GAS  /tmp/ccNMEBpy.s 			page 25


 705              	.LVL33:
 242:Core/Src/timers.c ****   if (HAL_TIM_OC_ConfigChannel(&htim5, &sConfigOC, TIM_CHANNEL_1) != HAL_OK)
 706              		.loc 1 242 6 view .LVU224
 707 00a2 88B9     		cbnz	r0, .L56
 708              	.L43:
 251:Core/Src/timers.c **** }
 709              		.loc 1 251 1 view .LVU225
 710 00a4 15B0     		add	sp, sp, #84
 711              		.cfi_remember_state
 712              		.cfi_def_cfa_offset 4
 713              		@ sp needed
 714 00a6 5DF804FB 		ldr	pc, [sp], #4
 715              	.L51:
 716              		.cfi_restore_state
 209:Core/Src/timers.c ****     Error_Handler();
 717              		.loc 1 209 5 is_stmt 1 view .LVU226
 718 00aa FFF7FEFF 		bl	Error_Handler
 719              	.LVL34:
 720 00ae C5E7     		b	.L44
 721              	.L52:
 214:Core/Src/timers.c ****     Error_Handler();
 722              		.loc 1 214 5 view .LVU227
 723 00b0 FFF7FEFF 		bl	Error_Handler
 724              	.LVL35:
 725 00b4 CBE7     		b	.L45
 726              	.L53:
 218:Core/Src/timers.c ****     Error_Handler();
 727              		.loc 1 218 5 view .LVU228
 728 00b6 FFF7FEFF 		bl	Error_Handler
 729              	.LVL36:
 730 00ba CEE7     		b	.L46
 731              	.L54:
 227:Core/Src/timers.c ****     Error_Handler();
 732              		.loc 1 227 5 view .LVU229
 733 00bc FFF7FEFF 		bl	Error_Handler
 734              	.LVL37:
 735 00c0 D8E7     		b	.L47
 736              	.L55:
 233:Core/Src/timers.c ****     Error_Handler();
 737              		.loc 1 233 5 view .LVU230
 738 00c2 FFF7FEFF 		bl	Error_Handler
 739              	.LVL38:
 740 00c6 DEE7     		b	.L48
 741              	.L56:
 244:Core/Src/timers.c ****     Error_Handler();
 742              		.loc 1 244 5 view .LVU231
 743 00c8 FFF7FEFF 		bl	Error_Handler
 744              	.LVL39:
 251:Core/Src/timers.c **** }
 745              		.loc 1 251 1 is_stmt 0 view .LVU232
 746 00cc EAE7     		b	.L43
 747              	.L58:
 748 00ce 00BF     		.align	2
 749              	.L57:
 750 00d0 00000000 		.word	htim5
 751 00d4 000C0040 		.word	1073744896
 752 00d8 00000000 		.word	.LANCHOR3
ARM GAS  /tmp/ccNMEBpy.s 			page 26


 753 00dc 00000000 		.word	.LANCHOR4
 754              		.cfi_endproc
 755              	.LFE337:
 757              		.section	.text.timer_us_delay,"ax",%progbits
 758              		.align	1
 759              		.global	timer_us_delay
 760              		.syntax unified
 761              		.thumb
 762              		.thumb_func
 763              		.fpu fpv4-sp-d16
 765              	timer_us_delay:
 766              	.LVL40:
 767              	.LFB329:
  59:Core/Src/timers.c **** {
 768              		.loc 1 59 1 is_stmt 1 view -0
 769              		.cfi_startproc
 770              		@ args = 0, pretend = 0, frame = 0
 771              		@ frame_needed = 0, uses_anonymous_args = 0
 772              		@ link register save eliminated.
  60:Core/Src/timers.c ****     __HAL_TIM_SET_COUNTER(&htim6,0);
 773              		.loc 1 60 5 view .LVU234
 774 0000 034B     		ldr	r3, .L61
 775 0002 1A68     		ldr	r2, [r3]
 776 0004 0023     		movs	r3, #0
 777 0006 5362     		str	r3, [r2, #36]
  61:Core/Src/timers.c ****     while ((__HAL_TIM_GET_COUNTER(&htim6))<us);
 778              		.loc 1 61 5 view .LVU235
 779              	.L60:
  61:Core/Src/timers.c ****     while ((__HAL_TIM_GET_COUNTER(&htim6))<us);
 780              		.loc 1 61 47 discriminator 1 view .LVU236
  61:Core/Src/timers.c ****     while ((__HAL_TIM_GET_COUNTER(&htim6))<us);
 781              		.loc 1 61 11 discriminator 1 view .LVU237
  61:Core/Src/timers.c ****     while ((__HAL_TIM_GET_COUNTER(&htim6))<us);
 782              		.loc 1 61 13 is_stmt 0 discriminator 1 view .LVU238
 783 0008 536A     		ldr	r3, [r2, #36]
  61:Core/Src/timers.c ****     while ((__HAL_TIM_GET_COUNTER(&htim6))<us);
 784              		.loc 1 61 11 discriminator 1 view .LVU239
 785 000a 8342     		cmp	r3, r0
 786 000c FCD3     		bcc	.L60
  62:Core/Src/timers.c **** }
 787              		.loc 1 62 1 view .LVU240
 788 000e 7047     		bx	lr
 789              	.L62:
 790              		.align	2
 791              	.L61:
 792 0010 00000000 		.word	htim6
 793              		.cfi_endproc
 794              	.LFE329:
 796              		.section	.text.timer_set_trigger_period,"ax",%progbits
 797              		.align	1
 798              		.global	timer_set_trigger_period
 799              		.syntax unified
 800              		.thumb
 801              		.thumb_func
 802              		.fpu fpv4-sp-d16
 804              	timer_set_trigger_period:
 805              	.LVL41:
ARM GAS  /tmp/ccNMEBpy.s 			page 27


 806              	.LFB330:
  64:Core/Src/timers.c **** void timer_set_trigger_period(uint16_t period){
 807              		.loc 1 64 47 is_stmt 1 view -0
 808              		.cfi_startproc
 809              		@ args = 0, pretend = 0, frame = 0
 810              		@ frame_needed = 0, uses_anonymous_args = 0
 811              		@ link register save eliminated.
  66:Core/Src/timers.c ****     (&htim2)->Instance->ARR = period;
 812              		.loc 1 66 5 view .LVU242
  66:Core/Src/timers.c ****     (&htim2)->Instance->ARR = period;
 813              		.loc 1 66 13 is_stmt 0 view .LVU243
 814 0000 014B     		ldr	r3, .L64
 815 0002 1B68     		ldr	r3, [r3]
  66:Core/Src/timers.c ****     (&htim2)->Instance->ARR = period;
 816              		.loc 1 66 29 view .LVU244
 817 0004 D862     		str	r0, [r3, #44]
  69:Core/Src/timers.c **** }
 818              		.loc 1 69 1 view .LVU245
 819 0006 7047     		bx	lr
 820              	.L65:
 821              		.align	2
 822              	.L64:
 823 0008 00000000 		.word	htim2
 824              		.cfi_endproc
 825              	.LFE330:
 827              		.section	.text.timer_set_discharge_period,"ax",%progbits
 828              		.align	1
 829              		.global	timer_set_discharge_period
 830              		.syntax unified
 831              		.thumb
 832              		.thumb_func
 833              		.fpu fpv4-sp-d16
 835              	timer_set_discharge_period:
 836              	.LVL42:
 837              	.LFB331:
  71:Core/Src/timers.c **** void timer_set_discharge_period(uint16_t period){
 838              		.loc 1 71 49 is_stmt 1 view -0
 839              		.cfi_startproc
 840              		@ args = 0, pretend = 0, frame = 0
 841              		@ frame_needed = 0, uses_anonymous_args = 0
 842              		@ link register save eliminated.
  73:Core/Src/timers.c ****     (&htim5)->Instance->ARR = period;
 843              		.loc 1 73 5 view .LVU247
  73:Core/Src/timers.c ****     (&htim5)->Instance->ARR = period;
 844              		.loc 1 73 13 is_stmt 0 view .LVU248
 845 0000 014B     		ldr	r3, .L67
 846 0002 1B68     		ldr	r3, [r3]
  73:Core/Src/timers.c ****     (&htim5)->Instance->ARR = period;
 847              		.loc 1 73 29 view .LVU249
 848 0004 D862     		str	r0, [r3, #44]
  76:Core/Src/timers.c **** }
 849              		.loc 1 76 1 view .LVU250
 850 0006 7047     		bx	lr
 851              	.L68:
 852              		.align	2
 853              	.L67:
 854 0008 00000000 		.word	htim5
ARM GAS  /tmp/ccNMEBpy.s 			page 28


 855              		.cfi_endproc
 856              	.LFE331:
 858              		.section	.text.timers_trigger_discarge_manually,"ax",%progbits
 859              		.align	1
 860              		.global	timers_trigger_discarge_manually
 861              		.syntax unified
 862              		.thumb
 863              		.thumb_func
 864              		.fpu fpv4-sp-d16
 866              	timers_trigger_discarge_manually:
 867              	.LFB332:
 108:Core/Src/timers.c **** {
 868              		.loc 1 108 1 is_stmt 1 view -0
 869              		.cfi_startproc
 870              		@ args = 0, pretend = 0, frame = 24
 871              		@ frame_needed = 0, uses_anonymous_args = 0
 872 0000 F0B5     		push	{r4, r5, r6, r7, lr}
 873              		.cfi_def_cfa_offset 20
 874              		.cfi_offset 4, -20
 875              		.cfi_offset 5, -16
 876              		.cfi_offset 6, -12
 877              		.cfi_offset 7, -8
 878              		.cfi_offset 14, -4
 879 0002 87B0     		sub	sp, sp, #28
 880              		.cfi_def_cfa_offset 48
 110:Core/Src/timers.c ****     HAL_TIM_PWM_Stop(&htim2, TIM_CHANNEL_3); 
 881              		.loc 1 110 5 view .LVU252
 882 0004 1C4D     		ldr	r5, .L71
 883 0006 0821     		movs	r1, #8
 884 0008 2846     		mov	r0, r5
 885 000a FFF7FEFF 		bl	HAL_TIM_PWM_Stop
 886              	.LVL43:
 111:Core/Src/timers.c ****     HAL_TIM_Base_Stop(&htim2);
 887              		.loc 1 111 5 view .LVU253
 888 000e 2846     		mov	r0, r5
 889 0010 FFF7FEFF 		bl	HAL_TIM_Base_Stop
 890              	.LVL44:
 115:Core/Src/timers.c ****     GPIO_InitTypeDef GPIO_InitStruct = {0};
 891              		.loc 1 115 5 view .LVU254
 115:Core/Src/timers.c ****     GPIO_InitTypeDef GPIO_InitStruct = {0};
 892              		.loc 1 115 22 is_stmt 0 view .LVU255
 893 0014 0024     		movs	r4, #0
 894 0016 0594     		str	r4, [sp, #20]
 116:Core/Src/timers.c ****     GPIO_InitStruct.Pin = GPIO_PIN_2;
 895              		.loc 1 116 5 is_stmt 1 view .LVU256
 116:Core/Src/timers.c ****     GPIO_InitStruct.Pin = GPIO_PIN_2;
 896              		.loc 1 116 25 is_stmt 0 view .LVU257
 897 0018 0427     		movs	r7, #4
 898 001a 0197     		str	r7, [sp, #4]
 117:Core/Src/timers.c ****     GPIO_InitStruct.Mode = GPIO_MODE_OUTPUT_PP;
 899              		.loc 1 117 5 is_stmt 1 view .LVU258
 117:Core/Src/timers.c ****     GPIO_InitStruct.Mode = GPIO_MODE_OUTPUT_PP;
 900              		.loc 1 117 26 is_stmt 0 view .LVU259
 901 001c 0126     		movs	r6, #1
 902 001e 0296     		str	r6, [sp, #8]
 118:Core/Src/timers.c ****     GPIO_InitStruct.Pull = GPIO_NOPULL;
 903              		.loc 1 118 5 is_stmt 1 view .LVU260
ARM GAS  /tmp/ccNMEBpy.s 			page 29


 118:Core/Src/timers.c ****     GPIO_InitStruct.Pull = GPIO_NOPULL;
 904              		.loc 1 118 26 is_stmt 0 view .LVU261
 905 0020 0394     		str	r4, [sp, #12]
 119:Core/Src/timers.c ****     GPIO_InitStruct.Speed = GPIO_SPEED_FREQ_LOW;
 906              		.loc 1 119 5 is_stmt 1 view .LVU262
 119:Core/Src/timers.c ****     GPIO_InitStruct.Speed = GPIO_SPEED_FREQ_LOW;
 907              		.loc 1 119 27 is_stmt 0 view .LVU263
 908 0022 0494     		str	r4, [sp, #16]
 120:Core/Src/timers.c ****     HAL_GPIO_Init(GPIOA, &GPIO_InitStruct);
 909              		.loc 1 120 5 is_stmt 1 view .LVU264
 910 0024 0DEB0701 		add	r1, sp, r7
 911 0028 4FF09040 		mov	r0, #1207959552
 912 002c FFF7FEFF 		bl	HAL_GPIO_Init
 913              	.LVL45:
 123:Core/Src/timers.c ****     HAL_GPIO_WritePin(GPIOA, GPIO_PIN_2, GPIO_PIN_SET);
 914              		.loc 1 123 5 view .LVU265
 915 0030 3246     		mov	r2, r6
 916 0032 3946     		mov	r1, r7
 917 0034 4FF09040 		mov	r0, #1207959552
 918 0038 FFF7FEFF 		bl	HAL_GPIO_WritePin
 919              	.LVL46:
 126:Core/Src/timers.c ****     HAL_Delay(100); // 1000 ms delay
 920              		.loc 1 126 5 view .LVU266
 921 003c 6420     		movs	r0, #100
 922 003e FFF7FEFF 		bl	HAL_Delay
 923              	.LVL47:
 128:Core/Src/timers.c ****     GPIO_InitStruct.Pin = GPIO_PIN_2;
 924              		.loc 1 128 5 view .LVU267
 128:Core/Src/timers.c ****     GPIO_InitStruct.Pin = GPIO_PIN_2;
 925              		.loc 1 128 25 is_stmt 0 view .LVU268
 926 0042 0197     		str	r7, [sp, #4]
 129:Core/Src/timers.c ****     GPIO_InitStruct.Mode = GPIO_MODE_AF_PP;
 927              		.loc 1 129 5 is_stmt 1 view .LVU269
 129:Core/Src/timers.c ****     GPIO_InitStruct.Mode = GPIO_MODE_AF_PP;
 928              		.loc 1 129 26 is_stmt 0 view .LVU270
 929 0044 0223     		movs	r3, #2
 930 0046 0293     		str	r3, [sp, #8]
 130:Core/Src/timers.c ****     GPIO_InitStruct.Pull = GPIO_NOPULL;
 931              		.loc 1 130 5 is_stmt 1 view .LVU271
 130:Core/Src/timers.c ****     GPIO_InitStruct.Pull = GPIO_NOPULL;
 932              		.loc 1 130 26 is_stmt 0 view .LVU272
 933 0048 0394     		str	r4, [sp, #12]
 131:Core/Src/timers.c ****     GPIO_InitStruct.Speed = GPIO_SPEED_FREQ_LOW;
 934              		.loc 1 131 5 is_stmt 1 view .LVU273
 131:Core/Src/timers.c ****     GPIO_InitStruct.Speed = GPIO_SPEED_FREQ_LOW;
 935              		.loc 1 131 27 is_stmt 0 view .LVU274
 936 004a 0494     		str	r4, [sp, #16]
 132:Core/Src/timers.c ****     GPIO_InitStruct.Alternate = GPIO_AF1_TIM2;
 937              		.loc 1 132 5 is_stmt 1 view .LVU275
 132:Core/Src/timers.c ****     GPIO_InitStruct.Alternate = GPIO_AF1_TIM2;
 938              		.loc 1 132 31 is_stmt 0 view .LVU276
 939 004c 0596     		str	r6, [sp, #20]
 133:Core/Src/timers.c ****     HAL_GPIO_Init(GPIOA, &GPIO_InitStruct);
 940              		.loc 1 133 5 is_stmt 1 view .LVU277
 941 004e 0DEB0701 		add	r1, sp, r7
 942 0052 4FF09040 		mov	r0, #1207959552
 943 0056 FFF7FEFF 		bl	HAL_GPIO_Init
ARM GAS  /tmp/ccNMEBpy.s 			page 30


 944              	.LVL48:
 136:Core/Src/timers.c ****     HAL_GPIO_Init(GPIOA, &GPIO_InitStruct);
 945              		.loc 1 136 5 view .LVU278
 946 005a 0DEB0701 		add	r1, sp, r7
 947 005e 4FF09040 		mov	r0, #1207959552
 948 0062 FFF7FEFF 		bl	HAL_GPIO_Init
 949              	.LVL49:
 139:Core/Src/timers.c ****     HAL_TIM_Base_Start(&htim2);  
 950              		.loc 1 139 5 view .LVU279
 951 0066 2846     		mov	r0, r5
 952 0068 FFF7FEFF 		bl	HAL_TIM_Base_Start
 953              	.LVL50:
 140:Core/Src/timers.c ****     HAL_TIM_PWM_Start(&htim2, TIM_CHANNEL_3);
 954              		.loc 1 140 5 view .LVU280
 955 006c 0821     		movs	r1, #8
 956 006e 2846     		mov	r0, r5
 957 0070 FFF7FEFF 		bl	HAL_TIM_PWM_Start
 958              	.LVL51:
 141:Core/Src/timers.c **** }
 959              		.loc 1 141 1 is_stmt 0 view .LVU281
 960 0074 07B0     		add	sp, sp, #28
 961              		.cfi_def_cfa_offset 20
 962              		@ sp needed
 963 0076 F0BD     		pop	{r4, r5, r6, r7, pc}
 964              	.L72:
 965              		.align	2
 966              	.L71:
 967 0078 00000000 		.word	htim2
 968              		.cfi_endproc
 969              	.LFE332:
 971              		.section	.text.timers_init_timers,"ax",%progbits
 972              		.align	1
 973              		.global	timers_init_timers
 974              		.syntax unified
 975              		.thumb
 976              		.thumb_func
 977              		.fpu fpv4-sp-d16
 979              	timers_init_timers:
 980              	.LFB333:
 144:Core/Src/timers.c **** void timers_init_timers(void){
 981              		.loc 1 144 30 is_stmt 1 view -0
 982              		.cfi_startproc
 983              		@ args = 0, pretend = 0, frame = 0
 984              		@ frame_needed = 0, uses_anonymous_args = 0
 985 0000 08B5     		push	{r3, lr}
 986              		.cfi_def_cfa_offset 8
 987              		.cfi_offset 3, -8
 988              		.cfi_offset 14, -4
 145:Core/Src/timers.c ****   MX_TIM2_Init(); // discharge
 989              		.loc 1 145 3 view .LVU283
 990 0002 FFF7FEFF 		bl	MX_TIM2_Init
 991              	.LVL52:
 146:Core/Src/timers.c ****   MX_TIM5_Init(); // trigger
 992              		.loc 1 146 3 view .LVU284
 993 0006 FFF7FEFF 		bl	MX_TIM5_Init
 994              	.LVL53:
 147:Core/Src/timers.c ****   MX_TIM3_Init();
ARM GAS  /tmp/ccNMEBpy.s 			page 31


 995              		.loc 1 147 3 view .LVU285
 996 000a FFF7FEFF 		bl	MX_TIM3_Init
 997              	.LVL54:
 148:Core/Src/timers.c ****   MX_TIM6_Init(); // us delay
 998              		.loc 1 148 3 view .LVU286
 999 000e FFF7FEFF 		bl	MX_TIM6_Init
 1000              	.LVL55:
 149:Core/Src/timers.c ****   MX_TIM17_Init(); // temperature measuring
 1001              		.loc 1 149 3 view .LVU287
 1002 0012 FFF7FEFF 		bl	MX_TIM17_Init
 1003              	.LVL56:
 151:Core/Src/timers.c ****   if (DEBUG){
 1004              		.loc 1 151 3 view .LVU288
 154:Core/Src/timers.c **** }
 1005              		.loc 1 154 1 is_stmt 0 view .LVU289
 1006 0016 08BD     		pop	{r3, pc}
 1007              		.cfi_endproc
 1008              	.LFE333:
 1010              		.section	.text.timers_start_timers,"ax",%progbits
 1011              		.align	1
 1012              		.global	timers_start_timers
 1013              		.syntax unified
 1014              		.thumb
 1015              		.thumb_func
 1016              		.fpu fpv4-sp-d16
 1018              	timers_start_timers:
 1019              	.LFB334:
 155:Core/Src/timers.c **** void timers_start_timers(void){
 1020              		.loc 1 155 31 is_stmt 1 view -0
 1021              		.cfi_startproc
 1022              		@ args = 0, pretend = 0, frame = 0
 1023              		@ frame_needed = 0, uses_anonymous_args = 0
 1024 0000 08B5     		push	{r3, lr}
 1025              		.cfi_def_cfa_offset 8
 1026              		.cfi_offset 3, -8
 1027              		.cfi_offset 14, -4
 156:Core/Src/timers.c ****   HAL_TIM_Base_Start(&htim2);
 1028              		.loc 1 156 3 view .LVU291
 1029 0002 0848     		ldr	r0, .L77
 1030 0004 FFF7FEFF 		bl	HAL_TIM_Base_Start
 1031              	.LVL57:
 157:Core/Src/timers.c ****   HAL_TIM_Base_Start(&htim3);
 1032              		.loc 1 157 3 view .LVU292
 1033 0008 0748     		ldr	r0, .L77+4
 1034 000a FFF7FEFF 		bl	HAL_TIM_Base_Start
 1035              	.LVL58:
 158:Core/Src/timers.c ****   HAL_TIM_Base_Start(&htim5);
 1036              		.loc 1 158 3 view .LVU293
 1037 000e 0748     		ldr	r0, .L77+8
 1038 0010 FFF7FEFF 		bl	HAL_TIM_Base_Start
 1039              	.LVL59:
 159:Core/Src/timers.c ****   HAL_TIM_Base_Start(&htim6);
 1040              		.loc 1 159 3 view .LVU294
 1041 0014 0648     		ldr	r0, .L77+12
 1042 0016 FFF7FEFF 		bl	HAL_TIM_Base_Start
 1043              	.LVL60:
 161:Core/Src/timers.c ****   HAL_TIM_Base_Start_IT(&htim17);
ARM GAS  /tmp/ccNMEBpy.s 			page 32


 1044              		.loc 1 161 3 view .LVU295
 1045 001a 0648     		ldr	r0, .L77+16
 1046 001c FFF7FEFF 		bl	HAL_TIM_Base_Start_IT
 1047              	.LVL61:
 163:Core/Src/timers.c **** }
 1048              		.loc 1 163 1 is_stmt 0 view .LVU296
 1049 0020 08BD     		pop	{r3, pc}
 1050              	.L78:
 1051 0022 00BF     		.align	2
 1052              	.L77:
 1053 0024 00000000 		.word	htim2
 1054 0028 00000000 		.word	htim3
 1055 002c 00000000 		.word	htim5
 1056 0030 00000000 		.word	htim6
 1057 0034 00000000 		.word	htim17
 1058              		.cfi_endproc
 1059              	.LFE334:
 1061              		.section	.text.HAL_TIM_PeriodElapsedCallback,"ax",%progbits
 1062              		.align	1
 1063              		.global	HAL_TIM_PeriodElapsedCallback
 1064              		.syntax unified
 1065              		.thumb
 1066              		.thumb_func
 1067              		.fpu fpv4-sp-d16
 1069              	HAL_TIM_PeriodElapsedCallback:
 1070              	.LVL62:
 1071              	.LFB335:
 166:Core/Src/timers.c **** {
 1072              		.loc 1 166 1 is_stmt 1 view -0
 1073              		.cfi_startproc
 1074              		@ args = 0, pretend = 0, frame = 0
 1075              		@ frame_needed = 0, uses_anonymous_args = 0
 166:Core/Src/timers.c **** {
 1076              		.loc 1 166 1 is_stmt 0 view .LVU298
 1077 0000 08B5     		push	{r3, lr}
 1078              		.cfi_def_cfa_offset 8
 1079              		.cfi_offset 3, -8
 1080              		.cfi_offset 14, -4
 167:Core/Src/timers.c ****   temp_convert_temperature();
 1081              		.loc 1 167 3 is_stmt 1 view .LVU299
 1082 0002 FFF7FEFF 		bl	temp_convert_temperature
 1083              	.LVL63:
 168:Core/Src/timers.c **** }
 1084              		.loc 1 168 1 is_stmt 0 view .LVU300
 1085 0006 08BD     		pop	{r3, pc}
 1086              		.cfi_endproc
 1087              	.LFE335:
 1089              		.section	.text.timers_start_pwm,"ax",%progbits
 1090              		.align	1
 1091              		.global	timers_start_pwm
 1092              		.syntax unified
 1093              		.thumb
 1094              		.thumb_func
 1095              		.fpu fpv4-sp-d16
 1097              	timers_start_pwm:
 1098              	.LFB336:
 171:Core/Src/timers.c **** void timers_start_pwm(void){
ARM GAS  /tmp/ccNMEBpy.s 			page 33


 1099              		.loc 1 171 28 is_stmt 1 view -0
 1100              		.cfi_startproc
 1101              		@ args = 0, pretend = 0, frame = 0
 1102              		@ frame_needed = 0, uses_anonymous_args = 0
 1103 0000 08B5     		push	{r3, lr}
 1104              		.cfi_def_cfa_offset 8
 1105              		.cfi_offset 3, -8
 1106              		.cfi_offset 14, -4
 173:Core/Src/timers.c ****   HAL_TIM_PWM_Start(&htim2, TIM_CHANNEL_3);
 1107              		.loc 1 173 3 view .LVU302
 1108 0002 0821     		movs	r1, #8
 1109 0004 0148     		ldr	r0, .L83
 1110 0006 FFF7FEFF 		bl	HAL_TIM_PWM_Start
 1111              	.LVL64:
 174:Core/Src/timers.c ****   if (DEBUG){
 1112              		.loc 1 174 3 view .LVU303
 179:Core/Src/timers.c **** }
 1113              		.loc 1 179 1 is_stmt 0 view .LVU304
 1114 000a 08BD     		pop	{r3, pc}
 1115              	.L84:
 1116              		.align	2
 1117              	.L83:
 1118 000c 00000000 		.word	htim2
 1119              		.cfi_endproc
 1120              	.LFE336:
 1122              		.global	temp
 1123              		.global	compareTrigValue
 1124              		.global	timInterPeriod
 1125              		.global	timTrigPeriod
 1126              		.global	timDiscPulse
 1127              		.global	timDiscPeriod
 1128              		.comm	htim17,76,4
 1129              		.comm	htim16,76,4
 1130              		.comm	htim6,76,4
 1131              		.comm	htim5,76,4
 1132              		.comm	htim3,76,4
 1133              		.comm	htim2,76,4
 1134              		.section	.bss.temp,"aw",%nobits
 1135              		.align	2
 1138              	temp:
 1139 0000 00000000 		.space	4
 1140              		.section	.data.compareTrigValue,"aw"
 1141              		.align	2
 1142              		.set	.LANCHOR4,. + 0
 1145              	compareTrigValue:
 1146 0000 27000000 		.word	39
 1147              		.section	.data.timDiscPeriod,"aw"
 1148              		.align	2
 1149              		.set	.LANCHOR1,. + 0
 1152              	timDiscPeriod:
 1153 0000 BD000000 		.word	189
 1154              		.section	.data.timDiscPulse,"aw"
 1155              		.align	2
 1156              		.set	.LANCHOR2,. + 0
 1159              	timDiscPulse:
 1160 0000 8B000000 		.word	139
 1161              		.section	.data.timInterPeriod,"aw"
ARM GAS  /tmp/ccNMEBpy.s 			page 34


 1162              		.align	2
 1163              		.set	.LANCHOR0,. + 0
 1166              	timInterPeriod:
 1167 0000 09000000 		.word	9
 1168              		.section	.data.timTrigPeriod,"aw"
 1169              		.align	2
 1170              		.set	.LANCHOR3,. + 0
 1173              	timTrigPeriod:
 1174 0000 2B010000 		.word	299
 1175              		.text
 1176              	.Letext0:
 1177              		.file 2 "/usr/lib/gcc/arm-none-eabi/9.2.1/include/stdint.h"
 1178              		.file 3 "Drivers/CMSIS/Include/core_cm4.h"
 1179              		.file 4 "Drivers/CMSIS/Device/ST/STM32G4xx/Include/system_stm32g4xx.h"
 1180              		.file 5 "Drivers/CMSIS/Device/ST/STM32G4xx/Include/stm32g474xx.h"
 1181              		.file 6 "Drivers/STM32G4xx_HAL_Driver/Inc/stm32g4xx_hal_def.h"
 1182              		.file 7 "Drivers/STM32G4xx_HAL_Driver/Inc/stm32g4xx_hal_gpio.h"
 1183              		.file 8 "Drivers/STM32G4xx_HAL_Driver/Inc/stm32g4xx_hal_dma.h"
 1184              		.file 9 "Drivers/STM32G4xx_HAL_Driver/Inc/stm32g4xx_hal_flash.h"
 1185              		.file 10 "Drivers/STM32G4xx_HAL_Driver/Inc/stm32g4xx_hal_tim.h"
 1186              		.file 11 "Drivers/STM32G4xx_HAL_Driver/Inc/stm32g4xx_hal_uart.h"
 1187              		.file 12 "Drivers/STM32G4xx_HAL_Driver/Inc/stm32g4xx_hal.h"
 1188              		.file 13 "Drivers/STM32G4xx_HAL_Driver/Inc/stm32g4xx_hal_tim_ex.h"
 1189              		.file 14 "Core/Inc/main.h"
 1190              		.file 15 "Core/Inc/temperature.h"
ARM GAS  /tmp/ccNMEBpy.s 			page 35


DEFINED SYMBOLS
                            *ABS*:0000000000000000 timers.c
     /tmp/ccNMEBpy.s:18     .text.MX_TIM17_Init:0000000000000000 $t
     /tmp/ccNMEBpy.s:25     .text.MX_TIM17_Init:0000000000000000 MX_TIM17_Init
     /tmp/ccNMEBpy.s:80     .text.MX_TIM17_Init:000000000000002c $d
                            *COM*:000000000000004c htim17
     /tmp/ccNMEBpy.s:86     .text.MX_TIM3_Init:0000000000000000 $t
     /tmp/ccNMEBpy.s:92     .text.MX_TIM3_Init:0000000000000000 MX_TIM3_Init
     /tmp/ccNMEBpy.s:220    .text.MX_TIM3_Init:0000000000000080 $d
                            *COM*:000000000000004c htim3
     /tmp/ccNMEBpy.s:227    .text.MX_TIM6_Init:0000000000000000 $t
     /tmp/ccNMEBpy.s:233    .text.MX_TIM6_Init:0000000000000000 MX_TIM6_Init
     /tmp/ccNMEBpy.s:313    .text.MX_TIM6_Init:0000000000000048 $d
                            *COM*:000000000000004c htim6
     /tmp/ccNMEBpy.s:319    .text.MX_TIM2_Init:0000000000000000 $t
     /tmp/ccNMEBpy.s:325    .text.MX_TIM2_Init:0000000000000000 MX_TIM2_Init
     /tmp/ccNMEBpy.s:538    .text.MX_TIM2_Init:00000000000000ec $d
                            *COM*:000000000000004c htim2
     /tmp/ccNMEBpy.s:545    .text.MX_TIM5_Init:0000000000000000 $t
     /tmp/ccNMEBpy.s:551    .text.MX_TIM5_Init:0000000000000000 MX_TIM5_Init
     /tmp/ccNMEBpy.s:750    .text.MX_TIM5_Init:00000000000000d0 $d
                            *COM*:000000000000004c htim5
     /tmp/ccNMEBpy.s:758    .text.timer_us_delay:0000000000000000 $t
     /tmp/ccNMEBpy.s:765    .text.timer_us_delay:0000000000000000 timer_us_delay
     /tmp/ccNMEBpy.s:792    .text.timer_us_delay:0000000000000010 $d
     /tmp/ccNMEBpy.s:797    .text.timer_set_trigger_period:0000000000000000 $t
     /tmp/ccNMEBpy.s:804    .text.timer_set_trigger_period:0000000000000000 timer_set_trigger_period
     /tmp/ccNMEBpy.s:823    .text.timer_set_trigger_period:0000000000000008 $d
     /tmp/ccNMEBpy.s:828    .text.timer_set_discharge_period:0000000000000000 $t
     /tmp/ccNMEBpy.s:835    .text.timer_set_discharge_period:0000000000000000 timer_set_discharge_period
     /tmp/ccNMEBpy.s:854    .text.timer_set_discharge_period:0000000000000008 $d
     /tmp/ccNMEBpy.s:859    .text.timers_trigger_discarge_manually:0000000000000000 $t
     /tmp/ccNMEBpy.s:866    .text.timers_trigger_discarge_manually:0000000000000000 timers_trigger_discarge_manually
     /tmp/ccNMEBpy.s:967    .text.timers_trigger_discarge_manually:0000000000000078 $d
     /tmp/ccNMEBpy.s:972    .text.timers_init_timers:0000000000000000 $t
     /tmp/ccNMEBpy.s:979    .text.timers_init_timers:0000000000000000 timers_init_timers
     /tmp/ccNMEBpy.s:1011   .text.timers_start_timers:0000000000000000 $t
     /tmp/ccNMEBpy.s:1018   .text.timers_start_timers:0000000000000000 timers_start_timers
     /tmp/ccNMEBpy.s:1053   .text.timers_start_timers:0000000000000024 $d
     /tmp/ccNMEBpy.s:1062   .text.HAL_TIM_PeriodElapsedCallback:0000000000000000 $t
     /tmp/ccNMEBpy.s:1069   .text.HAL_TIM_PeriodElapsedCallback:0000000000000000 HAL_TIM_PeriodElapsedCallback
     /tmp/ccNMEBpy.s:1090   .text.timers_start_pwm:0000000000000000 $t
     /tmp/ccNMEBpy.s:1097   .text.timers_start_pwm:0000000000000000 timers_start_pwm
     /tmp/ccNMEBpy.s:1118   .text.timers_start_pwm:000000000000000c $d
     /tmp/ccNMEBpy.s:1138   .bss.temp:0000000000000000 temp
     /tmp/ccNMEBpy.s:1145   .data.compareTrigValue:0000000000000000 compareTrigValue
     /tmp/ccNMEBpy.s:1166   .data.timInterPeriod:0000000000000000 timInterPeriod
     /tmp/ccNMEBpy.s:1173   .data.timTrigPeriod:0000000000000000 timTrigPeriod
     /tmp/ccNMEBpy.s:1159   .data.timDiscPulse:0000000000000000 timDiscPulse
     /tmp/ccNMEBpy.s:1152   .data.timDiscPeriod:0000000000000000 timDiscPeriod
                            *COM*:000000000000004c htim16
     /tmp/ccNMEBpy.s:1135   .bss.temp:0000000000000000 $d
     /tmp/ccNMEBpy.s:1141   .data.compareTrigValue:0000000000000000 $d
     /tmp/ccNMEBpy.s:1148   .data.timDiscPeriod:0000000000000000 $d
     /tmp/ccNMEBpy.s:1155   .data.timDiscPulse:0000000000000000 $d
     /tmp/ccNMEBpy.s:1162   .data.timInterPeriod:0000000000000000 $d
     /tmp/ccNMEBpy.s:1169   .data.timTrigPeriod:0000000000000000 $d
ARM GAS  /tmp/ccNMEBpy.s 			page 36



UNDEFINED SYMBOLS
HAL_TIM_Base_Init
Error_Handler
HAL_TIM_SlaveConfigSynchro
HAL_TIMEx_MasterConfigSynchronization
HAL_TIM_OnePulse_Init
HAL_TIM_ConfigClockSource
HAL_TIM_PWM_Init
HAL_TIM_PWM_ConfigChannel
HAL_TIM_MspPostInit
HAL_TIM_OC_ConfigChannel
HAL_TIM_PWM_Stop
HAL_TIM_Base_Stop
HAL_GPIO_Init
HAL_GPIO_WritePin
HAL_Delay
HAL_TIM_Base_Start
HAL_TIM_PWM_Start
HAL_TIM_Base_Start_IT
temp_convert_temperature
